:10000000004000205D5E00009D5E00009F5E0000DD
:1000100000000000000000000000000000000000E0
:10002000000000000000000000000000A15E0000D1
:100030000000000000000000A35E0000A55E0000BC
:10004000A75E0000A75E000081620000A75E0000BE
:10005000A75E000000000000A75E0000A75E000091
:10006000A75E000059650000A75E0000A75E0000C3
:10007000A75E0000A75E0000A75E0000A75E00006C
:10008000A75E0000BD660000A75E0000A75E00003E
:10009000A75E0000A75E0000A75E0000A75E00004C
:1000A000A75E0000A75E0000000000000000000046
:1000B0000000000000000000000000000000000040
:1000C000054B0648033310B51B1A062B03D9044B06
:1000D000002B00D0984710BDA0020020A0020020F5
:1000E000000000000648074910B5091A8910CB0F17
:1000F0005918491003D0044B002B00D0984710BD6D
:10010000A0020020A00200200000000010B5074C53
:100110002378002B09D1FFF7D3FF054B002B02D02A
:10012000044800E000BF0123237010BDA00200209E
:100130000000000048AA0000094B10B5002B03D0B6
:100140000849094800E000BF08480368002B02D1B5
:10015000FFF7C8FF10BD064B002BF9D09847F7E713
:1001600000000000A402002048AA00009C02002019
:1001700000000000164B002B00D1144B9D4640227E
:1001800092029A1A924600218B460F461348144A4F
:10019000121A08F072F90F4B002B00D098470E4B43
:1001A000002B00D098470020002104000D000D48CE
:1001B000002802D00C4800E000BF08F01BF9200026
:1001C000290006F075F808F0EFF8C04600000800B6
:1001D000004000200000000000000000A0020020FD
:1001E000F42500200000000000000000012303406F
:1001F0000200181E04D1042A03D91068000900E087
:100200000020704710B50400FFF7F0FF0300002046
:1002100083420BD0013B9B00181DE2181279002A83
:1002200003D001338342F8D100E0180010BD012251
:10023000096810B5114201D0002903DA102000F03E
:1002400083F903E04910062002F0ACF810BD0968FC
:1002500010B5CB0701D5002903DA102000F074F99E
:1002600006E04910033189100022052002F09AF8B7
:1002700010BD70B50D68AB0728D1042D26D90F230A
:100280002A684E681340062B09D12800FFF7AEFFFD
:10029000012383421DDC9A00AE500133F9E7052BA0
:1002A00014D1F30703D4132000F04EF912E07610B6
:1002B000FF2EF8D82800FFF799FF2C1D230080009F
:1002C0002018984205D91E700133FAE70B2000F080
:1002D0003BF9002070BD70B50C681120E3072DD5E7
:1002E0004D68AB0729D1042D27D90F262B68641040
:1002F0001E40062E0BD1002C04DD2800FFF776FFF0
:10030000844201DD122019E0A400605918E0331F77
:10031000012B12D82800FFF769FF8000042E02D1BC
:100320002800FFF76FFF002CECDDA042EADB012381
:100330002C19E0784000184302E00B2000F004F98B
:1003400070BDF8B501230C6811201C422FD0032585
:100350004E6835402AD1042E28D90F233268641004
:100360008F681340062B0BD1002C04DD3000FFF703
:100370003DFF844201DD122019E0A400A75113E0E3
:10038000052B13D1002CF6DD3000FFF72FFF800086
:100390008442F0DC01231F4201D1132007E07F10CB
:1003A000FF2FFAD83419E770280002E00B2000F084
:1003B000CBF8F8BD086810B5830717D1042815D904
:1003C0000F2302681340062B02D1FFF70FFF0BE04B
:1003D000052B05D1FFF70AFFC0000123184308E0F1
:1003E000042B03D1FFF70EFF4000F6E70B2000F0CF
:1003F000ABF810BD012303400200181E01D05010BD
:1004000002E00D22014B1A707047C046BC0200206A
:10041000012303400200181E04D1042A03D91068E6
:10042000000900E00020704770B50D000400FFF7E0
:10043000EFFF86002800FFF7EBFF830000209E42BD
:100440000ED1231D9E1904351A009E4207D9297822
:100450001278013301358A42F6D0002000E00120F5
:1004600070BD0000F0B585B00393019002912D4E50
:100470002D4B002A02D002223270013A00251A6068
:100480001B68F554019B9D424ADA029AAB00D05892
:10049000254B1C68C8239B0037191C1B01231842DD
:1004A00002D04310214A1FE0214A002802D004282C
:1004B00005D1204A2100380008F0A6FB18E00428E6
:1004C00010D90F2302681340042B04D101F0A6FFBA
:1004D000194A030008E0062B05D1FFF799FF174AD8
:1004E000030001E00123164A2100380008F08CFBCC
:1004F000300008F0EFFB039B0B4A002B01D110608A
:100500000CE0019B013B9D42F9DA0E4B9842F6DC70
:10051000431C1360202232540022F2540135B1E70B
:1005200005B0F0BDC8020020C4020020F999000007
:10053000CC990000D2990000C5A30000D799000013
:10054000E89900001F030000014B1870002070475D
:10055000BC02002070B501F07FFD094C0100251D93
:100560001F22280008F0BDFB280008F0B3FB04237D
:1005700004308008000118432060200070BDC04690
:10058000E8050020C368F0B59D00836889B05D1957
:10059000030018330693036903909E00069B9F197E
:1005A00043699E000193069B9E19CB4B1B78002B41
:1005B0000FD17F222B68C9491C1213409B005B5846
:1005C00001960435029235E0C34B1B78002B29D0ED
:1005D000019E039BC04C9B6821780193EA1A039B00
:1005E00092109B7812021A43039B587803F0E8FBA1
:1005F0000023039A2370137001960497039B069AB5
:100600009B680293ED1A039BAD10DD60049B9F1A5B
:10061000039BBF101F61019B9B1A039A9B105361A0
:1006200009B0F0BD2B68029A1C121340AB4A9B0024
:100630009B5804359F46039B587803F0B9FB002371
:10064000039A1370D9E7069B3A1DD11AA24BDB29F6
:1006500003DD1A22019E1A70BBE71B783C60002B59
:1006600002D0019E1700B4E72B6802991C120B40C0
:100670009A499B005B5817000435DBE7069B3A1D3F
:10068000D11A954BDB2903DD1A22019E1A70A0E7CF
:1006900028681B78291D3860002B03D0019E1700A5
:1006A0000D0096E76B6802991C120B408B499B006A
:1006B0005B5817000835BDE7069B3A1DD11A864BDB
:1006C000DB2903DD1A22019E1A7082E7A4001B7841
:1006D0002C193C60002B02D0019E170079E72B6893
:1006E00002991C120B407D499B005B581700043592
:1006F000A0E7069B3A1DD11A774BDB2903DD1A22AE
:10070000019E1A7065E77648A40021581B7839606D
:10071000002B02D0019E17005BE72B6802991C1288
:100720000B406E499B005B581700043582E7043F7D
:100730006B4B3A68A400E250674B1B78002B01D04A
:10074000019E46E72B68029A1C121340634A9B00E5
:100750009B5804356EE7624BA600F058FFF74AFE3F
:10076000043F04003868FFF745FE241801205C4B65
:1007700064000443F450584B1B78002B01D0019EB9
:1007800027E72B68029A1C121340544A9B009B587F
:1007900004354FE7069B3A1DD11A4F4BDB2903DD89
:1007A0001A22019E1A7014E70198069C0121A042AA
:1007B00002D901000C3909681B783960002B02D07E
:1007C000019E170005E72B6802991C120B40434954
:1007D0009B005B58170004352CE7069B3A1DD11A85
:1007E0003D4BDB2903DD1A22019E1A70F1E60199C7
:1007F000069881420AD90B000C3B1B6839495B10F3
:100800006418E41A019BA400E35802E0182119704F
:1008100000233B60304B1B78002B02D0019E170059
:10082000D7E62B6802991C120B402C499B005B58A1
:1008300017000435FEE6019B069A93420CD90C3B47
:100840001968284B3E1FE3184910591A3268019B5A
:100850008900CA50370002E018221F4B1A701E4B45
:100860001B78002B01D0019EB3E62B68029A1C1264
:1008700013401A4A9B009B580435DBE6019B069AFD
:10088000934220D9174B3E1FE318019C04930C3C64
:100890002368049A5B10D31A019A9B009858FFF7BB
:1008A000A9FD07903068FFF7A5FD2468049B64103C
:1008B0001C1B079BA4001F1801207F00019B0743FE
:1008C000E750370002E01822034B1A70024B1B78E6
:1008D000002B09D0019E7CE6BC0200200C9A00008F
:1008E00038230020FDFFFF3F2B68029A1C121340A3
:1008F000CD4A9B009B5804359CE6069B3A1DD11AB5
:10090000CA4BDB2903DD1A22019E1A7061E60199A8
:10091000A40061581B783960002B02D0019E17009B
:1009200057E62B6802991C120B40BF499B005B588D
:10093000170004357EE6043F019B3A68A400E250AC
:10094000BA4B1B78002B01D0019E42E62B68029A1D
:100950001C121340B44A9B009B5804356AE6019B65
:10096000A4001C192368043F38685E10FFF742FD9D
:1009700036180120AD4B76001B7806432660002B0D
:1009800001D0019E25E62B68029A1C121340A64A4C
:100990009B009B5804354DE6069BA4003F1BA34CCF
:1009A000BB420DD82378002B01D0019E11E62B68A5
:1009B000029A1C1213409C4A9B009B58043539E64E
:1009C0009B4801F09FFC2378002B01D0019E00E69C
:1009D0002B68029A1C121340934A9B009B580435C3
:1009E00028E6A300ED18002C00DA06E68F4B1B78F2
:1009F000002B01D0019EECE52B68029A1C121340DB
:100A0000894A9B009B58043514E63B1F04931B68DE
:100A10000793042B04D1A300ED18002C00DAEDE5B8
:100A2000824B1B78002B02D0019E049FD1E52B68DE
:100A3000029A1C1213407C4A9B009B58049F043569
:100A4000F8E53B1F04931B68042B06D0A200AD18E9
:100A5000002C02DA002B00D1D0E5744B1B78002B60
:100A600002D0019E049FB4E52B68029A1C12134029
:100A70006D4A9B009B58049F0435DBE53A1F1368C1
:100A80005B10013B002B07DD01215B00A4000B4341
:100A900004972D191360B1E5644B17001B78002BE8
:100AA00001D0019E95E52B68029A1C1213405E4A04
:100AB0009B009B580435BDE53A00069B0C32D31AC7
:100AC000DB2B04DD1A22594B019E1A7081E5FF23AE
:100AD00061005B000B4001210B433B60039B0698C8
:100AE0009B6824120493ED1A039BAD109B782D0292
:100AF0001D43019B8D401B1A9B108B400B43BB6019
:100B0000039B0D437D609C70E4B24A4BE400039963
:100B1000E35816008B6045490978002903D0083353
:100B20001D00170055E51D0002999B680C351C122D
:100B30000B403D499B005B58019217007AE53B1F33
:100B40001C68069A019B93422AD104970A20E30766
:100B500016D4A3070DD1042C0BD90F232268134000
:100B6000042B06D1200001F059FC08F0B3F8063040
:100B700006E00720042C03D0002C01D08020800048
:100B8000643002F019FE002801D1043D36E5039BD4
:100B90002100587803F026F90023039A13702DE5FD
:100BA000019B019A0C3B1B6803995B109B005B4205
:100BB0001E00D3180C3B1C601300083B1B68083E4A
:100BC00097195A108A70D2B21A49D2005B00555850
:100BD0009B0A039A9B009560ED18019B043B1E68DD
:100BE000069B7610B6009E19104B1B78002B00D088
:100BF000EFE42B68029A1C1213400B4A9B009B588F
:100C00000196043516E53B1F1868FFF7F3FBA400B7
:100C100006003F1B1E2831DC002816DC034B1B7826
:100C2000002B09D0019ED4E40C9A0000BC020020E5
:100C3000FC990000401B00202B68029A1C121340F4
:100C4000C54A9B009B580435F4E401F0EBF9033EE0
:100C5000361801F0E7F9C14B801B9842F9D8C04B18
:100C60001B78002B01D0019EB3E42B68029A1C1262
:100C70001340B94A9B009B580435DBE40123039AD7
:100C8000137001F0CFF9039B0A3886195E60B4E453
:100C90003B1F1868FFF7AEFBA40004903F1B002821
:100CA0000EDCAF4B1B78002B01D0019E91E42B682A
:100CB000029A1C121340A84A9B009B580435B9E4C1
:100CC000A84B049A019E9A4203DD1D22A44B1A7080
:100CD0007FE40123039A137001F0A4F9FA23049A24
:100CE0009B005343039A0A3B1B18536085E4A300FF
:100CF000FF1A002320001A003900FFF7B3FB9A4EB9
:100D00009A4C3168200002F033FF3168200003F074
:100D100070F83168200001F055FC914B1B78002BD6
:100D200001D0019E55E42B68029A1C1213408A4A96
:100D30009B009B5804357DE4894BA4001B783F1B26
:100D4000002B01D0019E44E42B68029A1C12134030
:100D5000814A9B009B5804356CE4039802F090FD97
:100D60007F4B1B78002B01D0019E32E42B68029A46
:100D70001C121340784A9B009B5804355AE43B1FD1
:100D80001868002824D1083B1868C30701D5401013
:100D900017E083070FD104280DD90F2302681340F1
:100DA000062B02D1FFF734FB0BE0052B03D1FFF735
:100DB0002FFB800005E01922694B019E1A70FFF796
:100DC00008FC3A0001214300083A0B43136001E09C
:100DD00040100138002832DD012243001343391F3F
:100DE0000B603B00083B1B681341181A3B000C3B8F
:100DF0001B68134203D08018A400904015E09907A7
:100E000017D1042B15D90F211E683140062906D1B0
:100E100001308000C358019AA400A35010E00529B6
:100E200007D118180079A4004000019B1043E0503E
:100E300006E019224A4B019E1A70FFF7CAFB0435DF
:100E4000474B1B78002B02D0019EFFF7C2FB2B689B
:100E5000029A1C121340404A9B009B580435FFF72E
:100E6000E9FBA300069AFB189B1ADB2B01DC01228D
:100E700005E01A223A4B019E1A70FFF7AAFB631E87
:100E8000002C03DD3A601C000437F8E7344B1B7874
:100E9000002B02D0019EFFF79CFB2B68029A1C12CC
:100EA00013402D4A9B009B580435FFF7C3FB069A5D
:100EB0003B1D9B1A2A4EDB2B04DD1A233370019E47
:100EC000FFF787FB019B069AA400934218D93B1FAA
:100ED0001868FFF78FFA002810DD019B0C3B1B6898
:100EE0005B1098420ADC9A07D31A1818204BC018D6
:100EF000019B8000C2583B1B1A6003E0202300E0E6
:100F000018233370164B3E1B1B78371D002B02D065
:100F1000019EFFF75EFB2B68029A1C1213400E4ADB
:100F20009B009B580435FFF785FBA3009C46F81AED
:100F3000002C04DC1C220A4B00261A7024E000213D
:100F400003685B1001268A008258164012D10D22D8
:100F5000034B1A7018E0C0460C9A00009F860100EF
:100F6000BC02002080EE3600C4020020C80200202F
:100F7000FCFFFF3F5210934200DD130001318C4211
:100F8000E0DC01265B001E4363460660FE1AD34B7D
:100F9000371D1B78002B02D0019EFFF71AFB2B6830
:100FA000029A1C121340CE4A9B009B580435FFF74F
:100FB00041FBA3009C46F81A002C04DC1C22C74B02
:100FC00000261A7015E0002103685B1001268A00D4
:100FD0008258164003D10D22C04B1A7009E05210FE
:100FE000934200DA130001318C42EFDC01265B00F2
:100FF0001E4363460660FE1AB84B371D1B78002B54
:1010000002D0019EFFF7E5FA2B68029A1C121340EA
:10101000B34A9B009B580435FFF70CFB3B00083B91
:101020001868FFF7E7F93B1F04901868FFF7E2F92B
:10103000049AA600BC1B0023824200DA043323601A
:10104000A64BBE1B1B78371D002B02D0019EFFF75D
:10105000C0FA2B68029A1C121340A14A9B009B58AD
:101060000435FFF7E7FAA300FE1A04933B00083BA0
:101070001868FFF7BFF93B1F04001868FFF7BAF9BB
:10108000E20FC317A04253419B003360049BFE1A3A
:10109000924B371D1B78002B02D0019EFFF799FA67
:1010A0002B68029A1C1213408D4A9B009B580435F2
:1010B000FFF7C0FA3B00083B18683B1F1968A30004
:1010C000884202D1FB1A042222E004281ED9012200
:1010D000104201D0114219D10326304215D10F23FD
:1010E00002681A40042A10D131420ED104290CD9C9
:1010F0000A681340042B08D1FFF796F9431E984164
:10110000A600BE1B8000306003E0A3000022FB1A93
:101110001A60724BA4001B783E1B371D002B02D0B7
:10112000019EFFF756FA2B68029A1C1213406C4A74
:101130009B009B580435FFF77DFA3B00083B18687D
:101140003B1F1968A300884202D1FB1A002223E04A
:1011500004281FD90122104201D011421AD10326BE
:10116000304216D10F2302681A40042A11D13142AD
:101170000FD104290DD90A681340042B09D1FFF7B8
:1011800053F9030058425841A600BE1B800030604E
:1011900003E0A3000422FB1A1A60504BA4001B7842
:1011A0003E1B371D002B02D0019EFFF712FA2B6861
:1011B000029A1C1213404A4A9B009B580435FFF7C1
:1011C00039FAA300FE1A04933B00083B1868FFF7A6
:1011D00011F93B1F04001868FFF70CF9E217C30F61
:1011E000844253419B003360049BFE1A3B4B371DE6
:1011F0001B78002B02D0019EFFF7EBF92B68029AB7
:101200001C121340364A9B009B580435FFF712FA14
:101210003B00083B1868FFF7EDF83B1F0490186887
:10122000FFF7E8F8049AA600BC1B0023824200DD09
:1012300004332360294BBE1B1B78371D002B02D0C3
:10124000019EFFF7C6F92B68029A1C121340244A2C
:101250009B009B580435FFF7EDF93B1F1B68A4006A
:10126000043B591E8B413A1B9B0013601B4B171DFF
:101270001B78002B02D0019EFFF7ABF92B68029A76
:101280001C121340164A9B009B580435FFF7D2F9F5
:10129000A300FC1A04933B00083B1868FFF7AAF868
:1012A0003B1F06001868FFF7A5F836180120049BBD
:1012B000760006432660FE1A084B371D1B78002B6C
:1012C00002D0019EFFF785F92B68029A1C12134089
:1012D000034A9B009B580435FFF7ACF9BC02002081
:1012E0000C9A0000A300FE1A04933B00083B186808
:1012F000FFF780F83B1F04001868FFF77BF8241AFB
:101300000120049B640004433460FE1AEA4B371D3D
:101310001B78002B02D0019EFFF75BF92B68029A25
:101320001C121340E54A9B009B580435FFF782F9D5
:10133000A300FC1A04933B00083B1868FFF75AF817
:101340003B1F06001868FFF755F846430120049B31
:10135000760006432660FE1AD74B371D1B78002BFC
:1013600002D0019EFFF735F92B68029A1C12134038
:10137000D24A9B009B580435FFF75CF93B1F186865
:10138000FFF738F8A30006000493FC1A002803D1E5
:101390001F22C94B1A700AE03B00083B1868FFF790
:1013A00029F8310005F02EFA012640000643049B7F
:1013B0002660FE1AC04B371D1B78002B02D0019E01
:1013C000FFF707F92B68029A1C121340BB4A9B00D7
:1013D0009B580435FFF72EF93B1F1868FFF70AF8F2
:1013E000A30006000493FC1A002803D11F22B24B6D
:1013F0001A700AE03B00083B1868FEF7FBFF31005B
:1014000005F0E6FA012649000E43049B2660FE1A09
:10141000A94B371D1B78002B02D0019EFFF7D9F88E
:101420002B68029A1C121340A44A9B009B58043557
:10143000FFF700F93B1F1868FEF7DCFFC317C01861
:1014400058400123400018439B4BA4001B783E1BCF
:101450003060371D002B02D0019EFFF7BAF82B68D1
:10146000029A1C121340954A9B009B580435FFF7C3
:10147000E1F8A300FE1A07933068012C03D1FEF7B0
:10148000B9FF049008E0FEF7B5FF04007068FEF7AE
:10149000B1FF0130031B0493049B002B01DC0123EB
:1014A000049307F063FB049905F092FA0C190121EB
:1014B000079B64000C433460FE1A7F4B371D1B787A
:1014C000002B02D0019EFFF784F82B68029A1C12B1
:1014D00013407A4A9B009B580435FFF7ABF8A300F2
:1014E000FE1A31002000049300F0AAFF049B306034
:1014F000FE1A714B371D1B78002B02D0019EFFF79F
:1015000068F82B68029A1C1213406C4A9B009B5887
:101510000435FFF78FF8A300FE1A04933B00083B45
:101520001868FEF767FF3B1F04001868FEF762FFAC
:1015300004400120049B640004433460FE1A5E4BA7
:10154000371D1B78002B02D0019EFFF742F82B6855
:10155000029A1C121340594A9B009B580435FFF70E
:1015600069F8A300FC1A04933B00083B1868FEF7D7
:1015700041FF3B1F06001868FEF73CFF06430120B1
:10158000049B760006432660FE1A4B4B371D1B78E2
:10159000002B02D0019EFFF71CF82B68029A1C1248
:1015A0001340464A9B009B580435FFF743F8A300BD
:1015B000FC1A04933B00083B1868FEF71BFF3B1F17
:1015C00006001868FEF716FF46400120049B7600CF
:1015D00006432660FE1A384B371D1B78002B02D0BD
:1015E000019EFEF7F6FF2B68029A1C121340334A45
:1015F0009B009B580435FFF71DF83B1F1868FEF74A
:10160000F9FEC0430123400018432B4BA4001B7874
:101610003E1B3060371D002B02D0019EFEF7D9FF24
:101620002B68029A1C121340244A9B009B580435D5
:10163000FFF700F8A300FE1A04933B00083B18686C
:10164000FEF7D8FE3B1F04001868FEF7D3FE844067
:10165000012364001C43049B3460FE1A164B371DA3
:101660001B78002B02D0019EFEF7B3FF2B68029A75
:101670001C121340114A9B009B580435FEF7DAFFF9
:10168000A300FE1A04933B00083B1868FEF7B2FE65
:101690003B1F04001868FEF7ADFE044101236400FF
:1016A0001C43049B3460FE1A034B371D1B78002B30
:1016B00006D0019EFEF78DFFBC0200200C9A0000B0
:1016C0002B68029A1C121340E94A9B009B58043570
:1016D000FEF7B0FF3B000C3B1868FEF78BFE3B00AB
:1016E000083B06001868FEF785FEF1170200C317D5
:1016F000300005F0BFF93B1F049005911868FEF714
:1017000079FE02000498059905F068F9012340006C
:101710001843D84BA4001B783E1B3060371D002BAC
:1017200002D0019EFEF755FF2B68029A1C1213404F
:10173000CF4A9B009B580435FEF77CFFA300FE1A9E
:10174000310020000493FEF772FD049B3060FE1A06
:10175000C84B371D1B78002B02D0019EFEF739FFC6
:101760002B68029A1C121340C14A9B009B580435F7
:10177000FEF760FFA300FE1A310020000493FEF77D
:1017800066FD049B3060FE1ABA4B371D1B78002B98
:1017900002D0019EFEF71DFF2B68029A1C12134017
:1017A000B34A9B009B580435FEF744FFA300FF1A81
:1017B00039002000FEF75DFDAE4B1B78002B02D0F8
:1017C000019EFEF706FF2B68029A1C121340A84ADE
:1017D0009B009B580435FEF72DFFA300FE1A310035
:1017E00020000493FEF777FD049B3060FE1AA14BA6
:1017F000371D1B78002B02D0019EFEF7EAFE2B68F6
:10180000029A1C1213409A4A9B009B580435FEF71B
:1018100011FFA300FF1A39002000FEF792FD954B3F
:101820001B78002B02D0019EFEF7D3FE2B68029A94
:101830001C1213408E4A9B009B580435FEF7FAFE9B
:10184000A300FE1A310020000493FEF7B3FD049BB1
:101850003060FE1A874B371D1B78002B02D0019E8B
:10186000FEF7B7FE2B68029A1C121340804A9B00B9
:101870009B580435FEF7DEFE069A3B1D04937D4C13
:101880009B1ADB2B04DD1A23019E2370FEF7A1FEB9
:1018900000F0D2FB01234000184323783860002B6E
:1018A00003D0019E049FFEF794FE2B68029A1C123F
:1018B00013406F4A9B009B58049F0435FEF7BAFE05
:1018C000069A3B1D04936B4C9B1ADB2B04DD1A23F9
:1018D000019E2370FEF77DFE00F0A4FB664B4000E6
:1018E00018400123184323783860002B03D0019E51
:1018F000049FFEF76EFE2B68029A1C1213405C4A8E
:101900009B009B58049F0435FEF794FEA300FB1A2E
:101910000493012320001A000499FEF7A3FD574CFD
:101920002068643001F048FF002816D0039B21682E
:101930005A78534802F06BFA15E0A300FB1A04939F
:101940002000012300220499FEF78CFD4B4C2068F7
:10195000643001F031FF002802D1043DFEF74DFE56
:10196000474802F063F80123039A137000F05AFB12
:10197000444A23681268063353431818039B58607F
:10198000FEF73CFEFEF7E6FD3A4BA4001B783E1B3B
:101990003060371D002B02D0019EFEF71AFE2B6827
:1019A000029A1C121340324A9B009B580435FEF7E2
:1019B00041FEA4003E1B300000F074FB2D4B306054
:1019C0001B78371D002B02D0019EFEF702FE2B680C
:1019D000029A1C121340264A9B009B580435FEF7BE
:1019E00029FEA4003E1B300000F05EFB214B30605E
:1019F0001B78371D002B02D0019EFEF7EAFD2B68F5
:101A0000029A1C1213401A4A9B009B580435FEF799
:101A100011FEA4003E1B300000F048FB154B306067
:101A20001B78371D002B02D0019EFEF7D2FD2B68DC
:101A3000029A1C1213400E4A9B009B580435FEF775
:101A4000F9FDA4003F1B380000F04EFB094B1B784A
:101A5000002B02D0019EFEF7BCFD2B68029A1C12DF
:101A60001340034A9B009B580435FEF7E3FDC04634
:101A70000C9A0000BC020020FEFFFF7FC402002081
:101A8000C802002004000020A300FE1A310020003C
:101A9000049300F04BFB049B3060FE1AE64B371DAD
:101AA0001B78002B02D0019EFEF793FD2B68029A53
:101AB0001C121340E14A9B009B580435FEF7BAFD07
:101AC000A4003F1B380000F06BFBDB4B1B78002BA6
:101AD00002D0019EFEF77DFD2B68029A1C12134076
:101AE000D64A9B009B580435FEF7A4FD0121200037
:101AF00000F03EFBD04B1B78002B02D0019EFEF77E
:101B000068FD2B68029A1C121340CC4A9B009B581C
:101B10000435FEF78FFD0021200000F029FBC64BA5
:101B20001B78002B02D0019EFEF753FD2B68029A12
:101B30001C121340C14A9B009B580435FEF77AFDE6
:101B4000A4003E1B300000F049FBBB4B30601B780B
:101B5000371D002B02D0019EFEF73BFD2B68029A39
:101B60001C121340B54A9B009B580435FEF762FDDA
:101B7000A4003E1B300000F045FBAF4B30601B78EB
:101B8000371D002B02D0019EFEF723FD2B68029A21
:101B90001C121340A94A9B009B580435FEF74AFDCE
:101BA000A4003F1B380000F007FBA34B1B78002B61
:101BB00002D0019EFEF70DFD2B68029A1C12134005
:101BC0009E4A9B009B580435FEF734FDA4003F1B42
:101BD000380002F093FB984B1B78002B02D0019E3B
:101BE000FEF7F7FC2B68029A1C121340934A9B00E5
:101BF0009B580435FEF71EFDA4003E1B300002F08A
:101C000027FC8D4B30601B78371D002B02D0019EC6
:101C1000FEF7DFFC2B68029A1C121340874A9B00D8
:101C20009B580435FEF706FDA4003F1B380002F068
:101C300035FB814B1B78002B02D0019EFEF7C9FCBF
:101C40002B68029A1C1213407C4A9B009B58043557
:101C5000FEF7F0FCA4003E1B300002F035FB764B93
:101C600030601B78371D002B02D0019EFEF7B1FCBF
:101C70002B68029A1C121340704A9B009B58043533
:101C8000FEF7D8FCA300FF1A3900200000F008FF7F
:101C9000694B1B78002B02D0019EFEF79AFC2B6843
:101CA000029A1C121340654A9B009B580435FEF7AC
:101CB000C1FCA300FF1A3900200000F07BFD5E4B41
:101CC0001B78002B02D0019EFEF783FC2B68029A42
:101CD0001C121340594A9B009B580435FEF7AAFC7E
:101CE000A300FF1A3900200000F074FD524B1B784E
:101CF000002B02D0019EFEF76CFC2B68029A1C128E
:101D000013404E4A9B009B580435FEF793FCA300FA
:101D1000FF1A3900200000F085FD474B1B78002B8F
:101D200002D0019EFEF755FC2B68029A1C1213404C
:101D3000424A9B009B580435FEF77CFCA300FE1A28
:101D400031002000049302F0C4FB049B3060FE1AB3
:101D5000394B371D1B78002B02D0019EFEF739FC52
:101D60002B68029A1C121340344A9B009B5804357E
:101D7000FEF760FCA300FE1A31002000049302F07D
:101D8000C0FB049B3060FE1A2B4B371D1B78002BC9
:101D900002D0019EFEF71DFC2B68029A1C12134014
:101DA000264A9B009B580435FEF744FCA300FE1A0C
:101DB00031002000049302F066FB049B3060FE1AA1
:101DC0001D4B371D1B78002B02D0019EFEF701FC36
:101DD0002B68029A1C121340184A9B009B5804352A
:101DE000FEF728FCA300FE1A31002000049302F045
:101DF00063FB049B3060FE1A0F4B371D1B78002BD2
:101E000002D0019EFEF7E5FB2B68029A1C121340DC
:101E10000A4A9B009B580435FEF70CFCA300FF1AEE
:101E20003900200000F0DAFD034B1B78002B07D0AF
:101E3000019EFEF7CEFBC046BC0200200C9A0000BB
:101E40002B68029A1C121340414A9B009B58043590
:101E5000FEF7F0FBA300FF1A3900200000F00AFD96
:101E60003C4B1B78002B02D0019EFEF7B2FB2B6887
:101E7000029A1C121340364A9B009B580435FEF709
:101E8000D9FBA300FE1A31002000049300F01EFECF
:101E9000049B3060FE1A2F4B371D1B78002B02D09D
:101EA000019EFEF796FB2B68029A1C121340284AEB
:101EB0009B009B580435FEF7BDFBA300FF1A3900B9
:101EC000200000F073FD234B1B78002B02D0019EF5
:101ED000FEF77FFB2B68029A1C1213401C4A9B00E2
:101EE0009B580435FEF7A6FBA300FF1A390020001B
:101EF00001F0E4FB174B1B78002B02D0019EFEF78C
:101F000068FB2B68029A1C121340114A9B009B58D5
:101F10000435FEF78FFBA300FE1A31002000049366
:101F200001F0CCFB049B3060FE1A0A4B371D1B7876
:101F3000002B02D0019EFEF74CFB2B68029A1C126C
:101F40001340034A9B009B580435FEF773FBC046C1
:101F50000C9A0000BC0200200023F7B55A1E019223
:101F6000002B07DA00F0E6FD01F04EFE01F074FFF1
:101F70006423019300263000194B19688E4201DB5F
:101F8000019BEBE7174B1A680132914200DC0022FB
:101F9000F0241A601D68144F6C43E35D002B1DD0C4
:101FA000E419022B16D0012B0ED1002801D100F02C
:101FB00039F8F0226A430C4B0C499B185B68C31A32
:101FC0008B4201D80223BB54F0235D43064BEB5CEC
:101FD000022B03D12000FEF7D5FAD1E70136CBE77B
:101FE000C002002000000020E01100209F860100B8
:101FF0000020704700207047002070470020704785
:1020000001220020054B06491A6158500330043163
:1020100058508018083158501A60704700800040AE
:10202000040500000122034B1A64A822D20098582C
:102030007047C0460080004010B5FFF7F3FFFA215B
:10204000890004F055FB10BD10B50100014803F0F4
:10205000BFFE10BD6811002000487047149C0000AE
:102060001A20704770B5054E0400335C0D008B429A
:1020700002D004F0B7FA355570BDC0460C060020FA
:1020800070B50024064D635D012B05D100212000B1
:1020900004F0A8FA0023635501341A2CF2D170BD64
:1020A0000C0600200D20704735207047036870B57E
:1020B0005B100120052B12D8094A9B009C58094D42
:1020C0002B5D002B05D00021200004F08BFA0023AB
:1020D0002B55200004F030F901234000184370BD57
:1020E000409C00000C06002070B5036845685C1039
:1020F0006D1004D40B4B9D4202DD1D0000E0002555
:10210000192C0DD8084E335D012B05D0012120007C
:1021100004F068FA012333552900200004F09AF9ED
:1021200070BDC046FF0300000C0600200B6870B5B0
:102130005D10192D16D80024012804DD4C68043CDC
:10214000624262415400094E735D9C4204D02100FA
:10215000280004F047FA7455280004F077FA0423A5
:10216000012800D00023180070BDC0460C060020D6
:1021700070B504000D0019280ED8084E335C012BF1
:1021800004D0012104F02EFA012333552900200048
:102190004D1EA94104F044FA70BDC0460C06002053
:1021A000436810B5191F4A424A41006811004010A7
:1021B000FFF7DEFF10BD000037B56A46064B6946E3
:1021C00030CB30C203680220042B02D100F002FBA6
:1021D00001E000F027FB37BD0C9C000010B5084C57
:1021E000237D002B05D00021142004F0FBF90023EF
:1021F0002375142004F02AFA43425841800010BD90
:102200000C06002010B5084CA37D002B05D0002142
:10221000162004F0E7F90023A375162004F016FA3F
:1022200043425841800010BD0C06002070477047A3
:1022300010B5034A0421034801F02CFA10BDC04632
:1022400008000020DBA20000E12110B54902094886
:1022500003F09CFEFFF7D4FE0A2004F067F8002389
:10226000FF21054A995401331A2BFBD100F0B6FD2A
:1022700010BDC046681100200C060020F8B50B4EBA
:10228000070030000D0003F0C1FE041EAC4200DD6B
:102290002C003D00EB1B9C4205DD300003F0C0FE2E
:1022A00028700135F6E72000F8BDC046681100200F
:1022B00010B50100014803F071FE10BD6811002047
:1022C00010B5054C200003F077FEE1212000490203
:1022D00003F05CFE10BDC04668110020064B0120D3
:1022E0001A68064B06491A60C82200235200C850DB
:1022F00004339342FBD170473006002028060020AB
:102300003823002000B59BB00200054901A806F063
:10231000ADFC01A801F0A6FB01F09EFDFCE7C04664
:10232000589C000037B5184D04002868002801D0DB
:1023300006F090F8A400200006F082F8286000283B
:1023400001D1124809E001AB984208D2104B0219A2
:102350006B440193934202D20E48FFF7D3FF042847
:1023600002D808302860083C2B680B4A1C191360FF
:102370000A4BC8221C600120002309495200C850A2
:1023800004339342FBD137BD30060020699C000026
:102390001CFCFFFF999C0000280600202C06002052
:1023A0003823002070B50D4D0D4E2B684C1CA40039
:1023B00036681C19B44203D90A20FEF7C5F80BE0B1
:1023C0002C601D00AC4201D904C5FBE70F220901B6
:1023D000104008431860180070BDC0462806002051
:1023E0002C0600200322CB1C70B50C00D91711401D
:1023F000C9180500891000220420FFF7D3FF00232D
:10240000A34204DAE95CC21811710133F8E7E14331
:102410000023C917214041180B7170BD10B5830707
:1024200006D1042804D90F2304C81340042B03D079
:102430000E20FEF789F8014810BDC04632A2000008
:1024400010B503240868044006D1042804D90F23DA
:1024500002681340042B01D00E2011E0FFF7DEFFCD
:102460000378233B5942594110224018210006F0BD
:10247000DDFC80239B05C218054B9A4203D914202A
:10248000FEF762F802E001234000184310BDC04689
:10249000FFFFFF3F70B501240B680D001C4001D009
:1024A0005C1002E00D20FEF74FF8200004F022FC43
:1024B000264904F00BFB05F0E5FE02F0F7FA0022D6
:1024C000234B05F099F80023002204F0C9FA0124F7
:1024D0002B681C40002819D0002C01D05C1002E0B1
:1024E0000D20FEF731F8200004F004FC174904F039
:1024F000EDFA05F0C7FE02F0D9FA0022144B05F000
:102500007BF80022134B04F03DFC18E0002C01D0B6
:102510005C1002E00D20FEF717F8200004F0EAFB43
:102520000A4904F0D3FA05F0ADFE02F0BFFA00222A
:10253000074B05F061F80022064B05F0D7FA05F0CD
:1025400029FE01234000184370BDC046D30237392D
:102550000000D0400000E03F10B5034A02210348CC
:1025600001F098F810BDC04628000020049D00002E
:102570000020704710B51E20FDF7E6FF10BD10B516
:102580001E20FDF7E1FF10BD10B51E20FDF7DCFF9A
:1025900010BD10B51E20FDF7D7FF10BD10B51E20D1
:1025A000FDF7D2FF10BD10B51E20FDF7CDFF10BD09
:1025B00010B51E20FDF7C8FF10BD10B51E20FDF799
:1025C000C3FF10BD7047000010B5034A092103483E
:1025D00001F060F810BDC04638000020169D0000D4
:1025E0000123034A1360034A106898401843704758
:1025F0003C06002044060020F0B5EFF310810123D3
:10260000194083F31088134E134AB4461268013AF6
:102610009340124A1468124A1568124A002B15D0CA
:10262000166803420BD02660C046C046C046C0466E
:10263000C046C046C046C04616682E6004E06746E5
:102640003E601668084F3E605B08E7E781F310883C
:10265000F0BDC04608050050C8000020500600200C
:102660004C060020380600200C05005030B585B01F
:1026700001AD0C220649280005F0F6FE0024285D75
:1026800001210134FFF7EEFC0C2CF8D105B030BD70
:10269000A29D0000F0B53B4C85B0210003220C3117
:1026A000684605F0E1FE210001AE0F31092230003D
:1026B00005F0DAFEFFF7C0FC334B344CC01823683A
:1026C000984201D2002323602568002D3CD1775D1C
:1026D00001213800FFF7C6FC01350121380003F065
:1026E0009FFF092DF3D100256B465E5D012130006F
:1026F000FFF7B8FC01350021300003F091FF032DF6
:10270000F2D1C82080000138C046C046C046C0464D
:10271000C046C046C046C046C046C046C046C04689
:10272000F1D100210520FFF79DFC00256B4600211B
:10273000585D0135FFF796FC032DF7D1FFF77CFCC0
:1027400013302060002519E0FFF776FC2368002590
:10275000984213D3052003F0EFFD0D4B0D4EC0182A
:1027600001D4306000E035603068032104F04AF89D
:1027700000230125084A306023601360280005B05B
:10278000F0BDC046A29D00001027000034060020C6
:10279000C8FEFFFF440600203C06002010B50124BF
:1027A000044001D0441002E00D20FDF7CDFE2000D2
:1027B00010BD00000022054B10B51A60044B1B68C9
:1027C000934201D001F010FF002010BD4806002008
:1027D0008C10002070B508680D00FFF7DFFF0400C3
:1027E0006868FFF7DBFF631E0100042B14D8451E49
:1027F000042D11D805226A43D318012215009D40EB
:102800002B00064805682B430360054B1B68002B13
:1028100002D0200001F0E9FE002070BD4806002033
:102820008C10002070B508680D00FFF7B7FF04009A
:102830006868FFF7B3FF631E0100042B14D8451E20
:10284000042D11D805226A43D31801229A4013009F
:10285000064802689A43064B02601B68002B03D0AF
:102860000022200001F0C1FE002070BD48060020BB
:102870008C100020F0B5050085B008680C00FFF74B
:102880008DFF0390022D08DD6068FFF787FF0700CA
:10289000A068FFF783FF040001E00124270005235F
:1028A0006343053B0293012326000193231D9E42AF
:1028B00034DC3D003B1D9D422BDC731E042B23D8D2
:1028C0006B1E042B20D8029B039A591E019B4919A9
:1028D0001A40204B0AD001228A4019680A431A6024
:1028E0001D4B01221B68002B0ED009E001208840FF
:1028F0000100186888431860174B1B68002B03D031
:102900003100280001F071FE019B01355B0001934D
:10291000D0E7029B013605330293C7E73D1D042D26
:1029200015D8012C13D126003300AB40094A116899
:102930009943094B11601B68002B04D0781D0022BD
:10294000210001F052FE01340535062CECD10020A7
:1029500005B0F0BD480600208C10002010B5041E04
:1029600013DBFFF77DFB84420FDA094BA400E2582A
:1029700001239340074A08491360084A1160084A36
:1029800008491160084A136010BD1A24EDE7C046DB
:1029900068A50000380600200805005050060020F9
:1029A0004C0600200C050050180500500B6810B5AF
:1029B0000200D80701D5581001E001204042182339
:1029C000012A03DD4A68042A00D10833024A136051
:1029D000FFF7C4FF002010BDC80000202D4BF7B545
:1029E0001B680C00002B03D101204042FFF7B6FF0B
:1029F00001262468344219D0FF2263101802120401
:102A00001040FF22611212020A40DBB21043184349
:102A1000214B1B68202B06D1B440204BA40EA400F0
:102A2000E35800021843FFF7E7FD30E00325254097
:102A30002DD1042C2BD90F2322681340062B26D12D
:102A4000FF27130901933F04019B9D421FDAAB004E
:102A5000E3185A68324218D0531018023840FF2148
:102A600084460902501208406146DBB2084318430D
:102A7000094B1B68202B06D15200920E074B920087
:102A8000D35800021843FFF7B7FD0135DCE70020FB
:102A9000FEBDC04638060020C8000020309E000061
:102AA000086810B5C30703D5FFF778FE054B18601B
:102AB000054B1B68002B03D0024B186801F096FDF4
:102AC000002010BD480600208C1000200868F8B5D2
:102AD000C30702D5FFF762FE0BE0830726D1042867
:102AE00024D90F2203681A40042A1FD11B091DD0C4
:102AF00000790300203B5E2B18D8052200205343A9
:102B00000B4E9D18043AAB420CD0052110249F5D5A
:102B10003C4200D080180139520064100029F7D1DE
:102B20000133F0E701234000184300E00120F8BD25
:102B3000309F00007FB5A44E3368002B0BD1A34A11
:102B40001268002A07D1A24B1B68002B00D139E183
:102B5000FFF7A0FD36E19F4D2A68002A2AD19C4A42
:102B60001268002A07D0FFF795FD002800D129E15F
:102B7000FFF77CFD05E0954A1268002A01D1002B81
:102B8000F6D1924B19681A00002911D03468002C34
:102B90000ED101AD0C22904928001C6005F064FCA8
:102BA000285D00210134FFF75DFA0C2CF8D109E112
:102BB0003368136000210D2003F032FD00210E2048
:102BC00003F02EFD00210F2003F02AFD2E68012EB8
:102BD00056D0022E00D19CE0002E00D0ECE0013651
:102BE00031007A4C04202368994303F019FD042135
:102BF000236805200B405942594103F011FD102173
:102C0000236806200B405942594103F009FD8021F9
:102C1000236809010B40594259410C2003F000FD83
:102C20008021236809020B40594259410B2003F0CF
:102C3000F7FC8021236849020B40594259410A2080
:102C400003F0EEFC8021236889020B405942594170
:102C5000092003F0E5FC80212368C9020B4059429A
:102C60005941082003F0DCFC802321681B030B4042
:102C700059425941072003F0D3FC31000D2099E05F
:102C80000221524C072023680B405942594103F05E
:102C9000C7FC0820216801400B005942594103F04C
:102CA000BFFC80212368C9000B40594259410520CF
:102CB00003F0B6FC8021236849010B405942594179
:102CC000062003F0ADFC80212368C9010B40594266
:102CD0005941042003F0A4FC8021236889030B40A0
:102CE000594259410A2003F09BFC802321681B04B0
:102CF0000B4059425941092003F092FC31000C204D
:102D000003F08EFC31000B2003F08AFC31000E2012
:102D100050E020212D4C072023680B405942594197
:102D200003F07EFC4021236808200B4059425941A2
:102D300003F076FC8021236809200B405942594159
:102D400003F06EFC8021236849000B405942594131
:102D50000A2003F065FC8021236889000B4059425A
:102D600059410B2003F05CFC8021236889010B4052
:102D7000594259410C2003F053FC80212368490338
:102D80000B4059425941062003F04AFC8021236838
:102D9000C9030B4059425941042003F041FC8023F0
:102DA00021685B040B4059425941052003F038FC6F
:102DB00001210F2003F034FC2B680321581C03F081
:102DC00007FE29607FBDC04648060020400600205F
:102DD0003C06002054060020A29D0000012010B5F2
:102DE0004042FFF7BBFD0020FFF706FC10BD0000CE
:102DF00010B5034A0921034800F04CFC10BDC04641
:102E000080000020BA9D000030B502248025094BC7
:102E1000094AED009C505C59002CFCD0A124E40030
:102E2000884204D28025ED0018514019F8E70021AE
:102E3000995030BD00E001400405000010B50028A5
:102E400004D1C020B0214002890203E0B0208021DB
:102E50008002C902FFF7D8FF10BD002802D0B023BE
:102E60009B0201E0C0235B021B6800201A0E532A5C
:102E700001D11B02180A704730B501248025064A8B
:102E8000064BED00D4505459002CFCD001600021B9
:102E9000014AD15030BDC04600E0014004050000A9
:102EA00010B5002802D0B020800201E0C02040020E
:102EB000A6230902DB05090A1943FFF7DDFF10BD50
:102EC000F0B50124802503000F4F08000F49ED00E5
:102ED0007C507C59002CFCD09C46002810DD547896
:102EE00016789378240234431B0423431C00D378C0
:102EF00001381B062343644608C40432A446ECE7A9
:102F000000237B50F0BDC04600E0014004050000F6
:102F100070B505004B680A009C1C2100FFF7D0FF2C
:102F2000A000281870BD0000154B1B68002B04D0B2
:102F30008021B023C9029B0203E0B021C023890293
:102F40005B02002807D1191D5B6802001B0E522B83
:102F500014D10A0012E0002281420FD903681B0E2F
:102F6000522B0BD1436802339B00C318994205D9F9
:102F70001A68110E0022522900D11A001000704761
:102F80005808002070B50020FFF7CEFFFF2605008F
:102F9000002808D003681C143440FFF7C5FFDA2C62
:102FA000F6D10500F4E7280070BD00008022F0B5DE
:102FB0005200A1B00021654805F05FFA802200218F
:102FC0005200634805F059FA624C23681A000393D3
:102FD00053425A4110000492FFF730FF039B0594BF
:102FE000002B01D15C4C00E05C4C0020FFF7CAFFD5
:102FF000FF270500002D7CD02A68131412123A40D6
:103000003B4002921A000A3A092A42D84F4B029AD0
:10301000995C002968D11022514805F02EFA2E0043
:10302000336802991A123A40914217D11A143A4061
:103030000B2A06D0132A0CD00A2A0FD1484B1E6047
:103040000CE03B40022B09DC454A9B00D3185E6034
:1030500004E010220021424805F00FFA3000FFF78B
:1030600063FF061EDCD13E4B196800290FD02000FB
:10307000FFF74EFF04003B4E3168002903D02000CB
:10308000FFF746FF0400384B0436B342F4D12F4B10
:1030900027E01A00153A082A26D82D4A0299565CCC
:1030A000002E21D1152B00D12E00280003681A1400
:1030B0003A40152A03D01D2A07D1002605E0029ABE
:1030C0001B123B409A4200D10600FFF72DFF00285B
:1030D000ECD1002E04D020003100FFF719FF0400CE
:1030E0001B4B0121029A99542800FFF71DFF050090
:1030F00080E70398FFF7B1FE411C0498FFF7D0FE6C
:10310000059B1A4D049A2C601A60FFF7D9F8059BAD
:103110002C681B68002B02D0B0239B0201E0C02367
:103120005B026420A021E41A6043490203F06AFBB9
:10313000A0225202030000920D49220007A805F0C8
:1031400095FD07A800F08EFC21B0F0BD58070020C7
:10315000580600205808002004C002000480010026
:10316000C8240020CC240020D82400205C080020A3
:1031700018A10000F0B50020B7B00024FFF7D4FE7E
:10318000270005002600002D20D0FF226B6828684C
:103190009C460233FF1803120136134011009C4273
:1031A00000DA1C0002140A400392624601400192B8
:1031B0000091039A1C4904A805F058FD04A800F0EA
:1031C00051FC2800FFF7B0FE0500DCE7174D28682A
:1031D000FFF743FE3B00019000943200144904A81D
:1031E00005F044FD04A800F03DFC124B1C682B6860
:1031F000002B02D0B0239B0201E0C0235B026420BD
:10320000A021E41A6043490203F0FCFAA022520212
:10321000030000920849220004A805F027FD04A835
:1032200000F020FC37B0F0BD4EA10000580800208F
:1032300062A100005C08002033A1000070B50020EE
:10324000FFF70BFE04000120FFF707FE844200DABF
:1032500004000A4B1E687542754128001D60FFF787
:10326000EDFD002E01D0064B00E0064B064A28007B
:10327000611C1360FFF714FE70BDC04658080020A3
:103280000480010004C002005C080020F8B50020A2
:10329000FFF7E3FD07000120FFF7DFFD3E00224DB1
:1032A0000643224C0CD18021C020C9024002FFF706
:1032B000ABFD01213000FFF7F3FD2E601C4B2FE02A
:1032C000874208DD0023B0212B60194B890223605F
:1032D0002368002011E0012380212B60154BC902D7
:1032E0002360F5E71A68551C18D0120E522A07D130
:1032F00001205A68023292009B188B42F2D311E0EF
:10330000002800D023600C4C0C49200005F0DAFCAA
:103310002000FEF799FEFFF791FF04E0002802D09D
:10332000236000E02160F8BD580800205C08002000
:103330000480010004C002001425002097A10000B1
:10334000F0B585B0039203220333DC1714402A4EF4
:10335000E3189C10336801900291002B02D0802268
:10336000D20201E0B0229202244FA51C3B68AD00BE
:103370005B199A4217D2FFF719FE3368002B02D06F
:103380008022D20201E0B02292023B685B199A428D
:1033900009D21B4C1B49200005F094FC2000FEF7CD
:1033A00053FE002026E0029B3E681B06190C6B466C
:1033B0001A7BA423DB051343019A0B431104FF225C
:1033C0001204114019433000FFF756FD3300301D41
:1033D0000833210001933B60FFF74EFD002C04D021
:1033E0000A9A21000198FFF76BFD3000019B083D10
:1033F0005D193D6005B0F0BD580800205C08002054
:1034000014250020C0A1000010B5FFF7CFFD10BDAE
:1034100070B59AB0FFF73AFFFF22264CD200002188
:10342000200005F02AF80020FEF7D8FE042804D179
:103430000020FEF7E7FE042831D00020FFF7A2FDB0
:10344000FF25002600281AD003681A142A400A2AE9
:1034500008D11A122A40FF2A0ED0D200A1180B71EF
:10346000A05009E0132A07D11B122B40FF2B03D0D9
:10347000DB00E2181671E650FFF756FDE2E7FF2188
:103480000200C900235808305D1EAB41D2188842A3
:10349000F8D1094901A805F0E9FB01A802E0FFF70E
:1034A000CDFE064800F0DEFA054800F0DBFA1AB05F
:1034B00070BDC046401B0020E7A1000003A2000031
:1034C000FBA10000002070470120704700487047B2
:1034D000F02400200048704733F8FFFF10B504497E
:1034E000044805F0EFFB24230348036010BDC046E9
:1034F000C6A20000DC240020D82400200020704751
:10350000002070470020704700207047002070475F
:10351000002070470020704700207047002070474F
:1035200010B5034A0E21034800F0B4F810BDC046A0
:10353000CC000020CBA20000044A05491368C854FF
:1035400001339B059B0D13607047C046680C00203B
:1035500060080020114A70B51368114C984211DAC6
:10356000015D451CFA39012906D8AB4206DD211858
:10357000497801391F2901D92800EFE70100251AF0
:10358000461C02D10023136006E0665C6E540131D4
:103590008B42FADC181A106070BDC0466C0C00201B
:1035A000780C002010B5FEF73DFD064B1A689042DE
:1035B00001D200221A601B68C01A034B834280416B
:1035C000404210BD740C0020204E000010B5094C84
:1035D000094A2368126893420BD0084AD05CFEF770
:1035E00067FE002805D0236801339B059B0D2360EF
:1035F000EDE710BD80100020680C0020600800205E
:1036000010B50400064B074A1B6812689B1ADB437F
:103610009B059B0DA34202DAFFF7D8FFF2E710BD2E
:10362000680C002080100020F7B506000191151EDF
:103630002FD05768B800441C0630FFF7E1FFFB208D
:10364000FFF77AFF1C20FFF777FFF0B2FFF774FF58
:10365000E0B22412FFF770FFE0B2FFF76DFF6B4698
:103660001879FFF769FF0026BE4212DAB300EB18A3
:103670009C680136E0B2FFF75FFF2012C0B2FFF78F
:103680005BFF2014C0B2FFF757FF200EFFF754FF77
:10369000EAE7F7BD70B5074D2C68092C08DC0C2350
:1036A0006343054E01349851F31859609A602C60B9
:1036B00070BDC0468410002078250020F0B589B088
:1036C00004900E0001284BDD284B08680293830705
:1036D00009D1042807D90F2302681340042B02D113
:1036E000FEF79CFE0290214B70680393830709D17B
:1036F000042807D90F2302681340042B02D1FEF7D8
:103700008DFE039000271A4B1A4D1B680593059BED
:103710009F4225DA2B1F0299186805F0C9FA002884
:103720001BD12B686C6806930190019B069A93420B
:1037300013DA20680399079405F0BAFA08340028D0
:1037400007D131000498079B08315B68023898471D
:1037500009E0019B01330193E7E701370C35D6E718
:103760001B20FCF7F1FE09B0F0BDC04632A20000FC
:10377000841000207C25002010B5FFF739FBFEF7F0
:1037800057FDFEF7E9FEFEF71FFFFFF7C9FE00F049
:10379000A9FD00F02DFF10BD962210B512010021E9
:1037A000034804F06AFE0022024B1A6010BDC046B6
:1037B000E0110020C0020020064B074A1B68126877
:1037C0009B1ADB439B059B0D0122834200DC0022F8
:1037D00010007047680C002080100020F8B505002C
:1037E0000C0016001F1E0ED10320FFF7E5FF002876
:1037F00027D0FA20FFF7A0FEE8B2FFF79DFEE0B267
:10380000FFF79AFE1DE0501DFFF7D6FF002818D0E5
:10381000FB20FFF791FEE8B2FFF78EFEE0B2FFF764
:103820008BFEF0B2FFF788FE3012C0B2FFF784FEC5
:103830003C00E31B9E4204DD2078FFF77DFE01344F
:10384000F7E7F8BD70B50024F0250B4B1B689C42D0
:103850000EDA2A006243094BD3181A78002A05D0E1
:103860005978002311201A00FFF7B8FF0134ECE764
:10387000FFF792FF70BDC046C0020020E01100209B
:1038800070B5060001250C4CB44212D02378002BF1
:103890000AD0002361781A001120FFF79FFFF02261
:1038A0000021200004F0E9FD0135F0340B2DEBD1AF
:1038B00070BD024B1D60F7E7E0110020C002002040
:1038C0000123F3B50400FFB00D0010001A420DD023
:1038D00002AA1370431002A9537042121B0E401427
:1038E0008A700B71C8700B00052273E0032313402C
:1038F0001ED1042A1CD90F2201680A40042A17D1BC
:10390000023302AA1370FEF789FD060005F0E2F902
:10391000F823FF33984200DD18000023834205DAC4
:1039200001335A1EB25C02A9CA54F7E7421C50E0A8
:10393000042801D0002809D1032302AA04381370F7
:103940004342434153701300022243E0002B45D110
:10395000042843D90F2102681140052912D10433EC
:1039600002A90B70F8231209FF3392009A4200DD7E
:103970001A00002393422BDA0133C118C97802AE32
:10398000F154F7E7062929D101390E0012095643EF
:103990000196F826019FFF36B7421FDC02AE317058
:1039A0000136934213DA0127013399004158394215
:1039B00001D0394100E00A49012737700F127170B8
:1039C000B7700F14090EF77031710536E9E7019AE7
:1039D000013202AB29002000FFF700FF7FB0F3BDEA
:1039E00019FCFFFF70B5F023050000240D4A1800F4
:1039F000604380184178A94203D001340A2CF6D1E3
:103A00000FE0F022002104F038FD074A1368013B63
:103A1000A34200D11460002329001A001120FFF7EF
:103A2000DDFE70BDE0110020C002002010B5B2B074
:103A300002236A460400137005F04CF9C72800DD24
:103A4000C7200023834205DA694601335A1EA25C6F
:103A5000CA54F7E7421C6B46FE211420FFF7BEFE56
:103A600032B010BD30B5B3B002236A460500137002
:103A700005F030F9041EC72C00DDC7240023A34243
:103A800005DA694601335A1EAA5CCA54F7E72000DA
:103A90003230FFF7B5FD621C6B46FF211420FFF7A3
:103AA0009DFE33B030BD0000F7B5234B06001B6808
:103AB000F020009300232149009A93420ADA020081
:103AC0005A438A185478B44202D11278002A31D16C
:103AD0000133F1E70024F0231A00624301920199B7
:103AE000164A55182F78002F06D001340A2CF3D12E
:103AF0001348FFF7B7FF1DE0F0223900280004F05B
:103B0000BCFC02230D4A0199EB6053540D4AF100AD
:103B10008A58009B6E70AE70AA602F616F61A342DD
:103B200002DC054B01341C60002331001A00102018
:103B3000FFF754FEF7BDC046C0020020E011002090
:103B400086A30000401B002010B5FFF77BFE002479
:103B5000064BE200D3181B79043B012B02D8E0B2DC
:103B6000FFF7A2FF0134FF2CF2D110BD401B002053
:103B7000F7B50E0000247F250190194BE200D11803
:103B80000979062901D0032926D1985883682B404A
:103B90001C2B21D1C3681A002A40042A1CD10269B7
:103BA0002A40192A18D11B0A01339B000C30C01877
:103BB000FEF734FC070005F08DF80023B0420BD16E
:103BC0009E4206DD019AF95CD25C914204D1013338
:103BD000F6E7E0B2FFF768FF0134FF2CCDD1F7BD67
:103BE000401B002070B505000024064BE200D318EE
:103BF0001B79AB4202D1E0B2FFF756FF0134FF2C34
:103C0000F3D170BD401B0020F7B5FEF70BFA514B06
:103C10001A68904201D200221A601A684E49821A2C
:103C20008A4200D894E01860FEF706FA071E00D119
:103C300001370020FEF7D2FA01900020FEF7E2FAE9
:103C4000019B0090454C464D002B17D02368002B5C
:103C50007AD12B682760002B72D0424B01261B784B
:103C6000002B06D10920FFF7BDFF3F4B1E703D4BD7
:103C700003E00720FFF7B6FF3B4B1E70009B002BB5
:103C800016D02B68002B13D123682F60002B22D075
:103C9000354B01261B78002B05D10920FFF7A2FF29
:103CA000314B1E7002E00820FFF79CFF2D4B1E7069
:103CB0002368002B0FD02C4E3278002A0BD19F4264
:103CC00000D227602368FB1A312B04D90720FFF7A5
:103CD00089FF012333702B68002B0FD0214E3278DF
:103CE000002A0BD19F4200D22F602B68FB1A312B88
:103CF00004D90820FFF776FF012333702368002BD7
:103D00000CD0019B002B09D1174E3378002B02D128
:103D10000720FFF767FF0023236033702B68002B19
:103D200016D0009B002B13D10E4B1A781C00002AD2
:103D300002D10820FFF756FF00232B60237007E015
:103D4000009B002BA0D1B3E7009A002A99D1B2E7DB
:103D5000F7BDC046600C00200F270000640C002057
:103D600078100020700C00207C10002037B5002453
:103D70000500FFF767FD01A80194FEF71DFA210079
:103D80002000FEF717FDFEF7D5FEFEF74FFAFEF70F
:103D90004EFAFFF723F8FEF773F9A54204D0FEF7B9
:103DA0009DFA0248FFF75EFE37BDC0469BA30000A8
:103DB000002310B501001A001120FFF70FFD10BD00
:103DC00007B56B46197069465A7013128B7013143D
:103DD000120ECB700A716B46010005221320FFF70B
:103DE000FDFC07BD10B50A0001001220FFF768FDB9
:103DF00010BD70B5050008000C003230FFF700FC64
:103E00002B00220000211B20FFF7E8FC70BD10B53D
:103E10000C000300110014202200FFF7DFFC10BD8E
:103E200070B506000020FFF77FF80024FF2500286A
:103E300010D003681A142A40152A05D11B122B40F2
:103E4000B34204D1040002E01D2A00D10024FFF790
:103E50006BF8ECE7200070BDF0B580279DB0FFF750
:103E6000B5FBB64DB64C2868FF00391A2018FEF78E
:103E700005FA2B680600C3182B60002B00D1D9E18E
:103E8000002E0DDD2868391A2018FEF7F7F92B6887
:103E900006001B182B60FEF7C5F8AA4B1860EFE769
:103EA0002378FA2B00D00CE12B68022B06DCFFF7FD
:103EB00079FB002800D1BDE10120B6E16078A5784A
:103EC0000238182800D9FAE002F008FC0D1E22265C
:103ED0002932F93D67F96F83D4E5F9F9F9F9F9F970
:103EE000F9F9F9F9F300FF2D00D1E8E02800FFF718
:103EF00079FD00229449EB005A50CB181A71290021
:103F00000092130013204DE02800FFF7CDFDD6E00E
:103F10002800FFF767FDD2E0FFF716FECFE0FFF7BE
:103F200091FC0020FFF722FF8848FFF79BFDC6E0C9
:103F3000632D00D9C3E0864BAA00D2582900152072
:103F4000FFF7BEFCBBE000242000FFF769FF071E5F
:103F500003D10134642CF7D1B1E0083004F0BAFE8B
:103F600006000530FFF74CFBFB20FFF7E5FA1D20AC
:103F7000FFF7E2FAE0B2FFF7DFFAF0B2FFF7DCFAA0
:103F80003012C0B2FFF7D8FA0025AE42E1DD7B194E
:103F9000187AFFF7D1FA0135F7E700211D200B0051
:103FA0000A000091FFF7CCF989E0FEF755F803AC61
:103FB000684A64210090684B200004F025FE02232B
:103FC0002000237004F086FE23000200002116204A
:103FD00073E000245C4AE300D558002D46D06B689E
:103FE0009E00701DFFF70CFB2B00002532000833EC
:103FF00021000120FFF7F2FB0020FEF795FF2E00C5
:104000002F0000281DD0FF2103681A120A40A24287
:1040100014D11A140A400B2A07D10B400DD0012BE2
:1040200009D0022B00D103E108E0132A06D10025B4
:104030002E002F0002E0060000E00700FEF774FFEC
:10404000DFE7002E04D0320001212000FFF7ECFA58
:10405000002D04D02A0002212000FFF7E5FA002FEE
:1040600004D03A0000212000FFF7DEFA0134FF2CD3
:10407000B0D124E00024FFF7E5FB220021000094EA
:104080002300DA20FFF75CF9FF222100D2002E483E
:1040900004F0F3F913E0012D02D1FFF76BF80EE005
:1040A000022D02D1FFF7B0F909E00120FFF75EFE13
:1040B00005E0002329001A001A20FFF78FFB0320D8
:1040C000B3E0FB2B00D0F7E62A68042A00DCEEE61A
:1040D0002679E078214B360206439E4200DDEBE66E
:1040E000331D9A4200DCE2E6E35CFE2B00D0E3E6FF
:1040F0006378A578711E1B2B5DD004D8012B08D0E6
:10410000082B2DD090E01D2B64D058D31E2B7BD0D4
:104110008AE0FF2D00D187E02800FFF763FC677974
:104120000634B31E290000943A000A20FFF708F96C
:10413000054BED00E8505D192F7175E06C0C002007
:10414000780C0020740C0020401B0020AAA3000063
:1041500038230020C1A30000BCA30000F603000028
:10416000632D61D86079022813D003281BD0012861
:104170005AD1A71D7A78A479BB78120222431B0476
:1041800013431A00FB78AD001B0613435B00034387
:104190000EE0002948DDB11EA01DFEF723F9264BD5
:1041A000AD00E85040E0A379AD005A1E93419B005A
:1041B000214AAB5038E0601DFFF7DAFC34E0627949
:1041C000FF2D31D0022A2FD80634B31E00942900C7
:1041D0000B2016E00B1E632B00DD6323002203A8D7
:1041E000934204DDA118497981540132F7E7D9439C
:1041F0000022C917194041180A70009029001520A3
:104200000133FFF79DF80FE0012D0DD100290BDDE3
:104210006379002B03D0322B02DD322300E02B0028
:1042200064225343054A1360701DFFF793F901E0C0
:10423000050003E71DB0F0BD382300200400002076
:104240000120704710B5064C200000F007FB05491F
:10425000200000F027FB0122034B1A6010BDC0466E
:10426000B0100020801A06008810002010B501212F
:104270000D20FDF7F7FE01210E20FDF7F3FE0021D2
:104280000F20FDF7EFFE044C200000F023FA102170
:10429000200000F03BFA10BD9C10002010B504680F
:1042A0000D20E30703D56410FF2C03D91720FCF77A
:1042B0004BF906E0FFF7DAFFE1B2024800F048FAF6
:1042C000002010BD9C10002010B5FFF7CFFF00218B
:1042D000034800F03DFA01234000184310BDC046DA
:1042E0009C10002010B5034A07210348FFF7D2F9BC
:1042F00010BDC0463C010020C8A30000F8B5012352
:1043000006681E4205D045681D4202D084681C42E2
:1043100001D10D2004E076106D10802E03D91520F8
:10432000FCF712F91DE01620FF2DF9D864101720B4
:10433000FF2CF5D80B4B1B68002B01D1FFF782FF38
:10434000094FF1B2380000F035FBE9B2380000F057
:1043500046FAE1B2380000F042FA380000F094FB6F
:104360000020F8BD88100020B0100020F7B501240F
:104370002300A04237DD0A68144234D01B4B55108D
:104380001B684C68002B01D1FFF75CFF0127184E1A
:10439000E9B2300000F00EFB3C4205D03C41300059
:1043A000E1B200F01CFA1AE00325254017D1042CD5
:1043B00015D90F2322681340062B10D1130901933E
:1043C000019B9D420BDAAB00E3185968394204D0D7
:1043D0004910C9B2300000F002FA0135F0E73000B0
:1043E00000F052FB00231800FEBDC04688100020DC
:1043F000B0100020144B70B51B6805000E00002B98
:1044000001D1FFF71FFF114CEDB22900200000F091
:10441000D1FAF1B2200000F0E2F90021200000F012
:10442000D5FA002801D040420CE0012229002000EA
:1044300000F0BBFA200000F0C8F90028FAD02000F4
:1044400000F0C8F970BDC04688100020B0100020F0
:1044500010B501240368234202D04168214201D1F2
:104460000D2004E058104910802803D91520FCF7CE
:104470006BF807E0FF2901D91620F8E7FFF7BAFF2C
:104480004000204310BD10B507211820FFF7B2FFF0
:104490007F2801DD0138FF3803007F3301DA7F20F8
:1044A000404264237F215843494202F0ABF9012383
:1044B00040424000184310BD10B508211820FFF7F6
:1044C00099FFC30F181801234010153040001843FE
:1044D00010BD10B505211820FFF78CFF7F2801DDE6
:1044E0000138FF3803007F3301DA7F204042642324
:1044F0007F215843494202F085F9012340001843C7
:1045000010BD10B503211820FFF774FF7F2801DDCF
:104510000138FF3803007F3301DA7F2040426423F3
:104520007F215843494202F06DF9012340001843AE
:1045300010BD0000F8B501263400B04236DD0F682A
:104540003E4233D04D68AB0730D1042D2ED90F2316
:104550002A681340062B29D1154B1B68002B01D16B
:10456000FFF770FE0024354204D12B681C09202C73
:1045700000D920240F4E7F10F9B22200300000F045
:1045800014FAA700EF19AF420DD0300000F01DF96A
:104590000028FAD0300000F01DF901234000184334
:1045A00068600435EFE70120640004432000F8BD93
:1045B00088100020B01000200020704700207047B5
:1045C000002070470020704700207047002070478F
:1045D000002070470020704700207047002070477F
:1045E00000207047002070477047704770470000F8
:1045F00010B5034A0C210348FFF74CF810BDC04624
:104600007401002009A4000010B5FDF71DFE064846
:10461000FDF788FEFFF7B0F80448FFF723FAFEF72E
:10462000F7FEFFF791FA10BDE20400007FA400003E
:1046300010B5FDF791FC10BD70B5002504AC2478D1
:104640000573A94205D10A4B0A4A23210A4803F0FF
:104650008BFE01600949920052589B0002715B5821
:104660008371A3005B58856043710223C37170BDE1
:10467000D4A4000097A40000E2A4000068A50000F4
:10468000037B002B04D143738373036101330373F2
:10469000704700001FB50191A02100240068C900E7
:1046A000D2B24450012A07D0A24203D0032A05D136
:1046B000042202E0022200E006221343034A835050
:1046C000034B019AC250012343501FBD5405000003
:1046D0002405000010B50400FFF7D2FFA1222368D3
:1046E000A179D20099506179064A20009950217928
:1046F00004329950044B19685A689B68FFF7CAFF47
:1047000010BDC0460C050000901000204BB2002BDD
:104710000CDB80233F290CD81F290CD80F290CD87B
:1047200007290CD803290CD81B060BE080239B0417
:1047300008E0DB0406E01B0504E05B0502E09B05E6
:1047400000E0DB050168014A8B507047240500003A
:104750000368074A99501A00FC32D1680029FCD03E
:10476000A321C90058580023C0B2D3607047C04687
:104770001C05000007B58022074BD2051A600022F5
:104780009A6002321A7111230E32009303490533E5
:104790000348FFF751FF07BD901000200030004094
:1047A0009C100020F8B505000E0017000024BC4244
:1047B00008D02B68315D1B6828009847002801D07D
:1047C0000134F4E72000F8BD704710B51C3001F04B
:1047D0002BFB10BD10B51C3001F018FB10BD70B5DF
:1047E000437E0D00002B05D06430040001F02BFB4C
:1047F000002801D0002004E02000290001F0F7FA91
:10480000012070BD10B51C3001F014FB10BD00007C
:10481000F7B50193FA23002504009B0083600D4B3C
:104820004560083303601C300F00160001F0D4FA15
:104830002000643001F0D0FA074AB600B35827616F
:104840006375019B20009B009B586576A576A37538
:10485000FEBDC04648A5000068A500000123A022B7
:10486000C375837D0C49C133FF33D2059B0099503A
:10487000437DC133FF339B009950CC210369074A24
:10488000490499500521243A9950817D0832995064
:10489000417D034A995070470C0600002405000032
:1048A0000C050000A02302690020DB00D05009485D
:1048B000814204D90848814204D9CD2103E0CC21AA
:1048C000490401E08021C904044811500521D15058
:1048D0007047C046A086010090D003002405000068
:1048E000F7B5050000200C00019382425CD0161E33
:1048F000402E00D940262F001C37380001F082FAE4
:10490000B1222B69D20080219C50012289005A508B
:10491000A97E002901D11A621A600024731E2A6937
:10492000A34206D1019B002B03D0802302219B00D0
:10493000D150012313621300FC33D968002902D13E
:10494000996A0029F9D0996A00290AD1D960A3236C
:10495000DB00D1583800C9B2013401F048FAA64250
:10496000DCD8019A2B69002A04D11A00FC32916A22
:1049700000290AD001210022AA7659611900FC31D0
:1049800088680028FCD08A6007E00121A976D961F7
:10499000D16C0029FCD00021D164FC339A6A002A32
:1049A00001D000229A62E0B2FEBD10B50123FFF7EC
:1049B00097FF10BD0300AC3310B5040019706430CC
:1049C00001F020FA0123637610BD0000F8B5002243
:1049D0000D0001004276AC31036904000878B12172
:1049E000C9005850802189005A5001321A629A60D9
:1049F00026006436300001F017FA00280ED030008F
:104A0000276901F003FA1E4BF8502369FC331A6A38
:104A1000002A0CD19A6A002AF9D008E02369002DF7
:104A20000AD11A00FC32916A002905D10EE09A6A77
:104A3000002AF3D11A62DBE701225A611A00FC3224
:104A400091680029FCD00021916006E00121D96124
:104A5000D16C0029FCD00021D1641A000020FC3266
:104A6000916A81420BD0074990625A5802305A50DD
:104A7000824204D0043A534253410230C01AF8BD76
:104A80001C050000C404000010B50121FFF79EFFC3
:104A900010BD000010B51323122202490248FFF78F
:104AA000B7FE10BD00400040B010002030B5214AD4
:104AB0004B0087B05B0893421EDD1F4A934205DD21
:104AC00002000B0003F012F807B030BD02AA00F09C
:104AD00035F803231840049A059B01281ED00228AC
:104AE00011D000281FD00298039900F02DFA8023DE
:104AF0001B069C466144E7E7002300220093002345
:104B000000F088FFE0E7012402980399009400F088
:104B100081FF80231B069C466144D5E702980399D8
:104B200000F012FAD0E7012402980399009400F0F3
:104B300071FFC9E7FB21E93FFFFFEF7FF0B54E466C
:104B400057464546E0B4DC4B4E0090B0170089460E
:104B500076089E4200DC81E0D84B9E4220DCD84A99
:104B6000002900DC89E1D74B02F0C0FFD54B0400DF
:104B70000D009E4200D18AE0D34AD44B02F0B6FF2A
:104B800002000B0020003A607B60290002F0AEFFBB
:104B9000CD4ACE4B02F0AAFFB860F960012066E072
:104BA000CB4B9E4200DC8DE0CA4B9E4265DCCA497D
:104BB00032158A46924453461B05F51A2900040013
:104BC00003F0E8FA03F01CFB02000B0020002900B0
:104BD0000A920B9302F08AFF0022C04B02F00CFDF8
:104BE0000290039103F0D6FA03F00AFB04000D00D3
:104BF00002000B00029803990C940D9502F076FFC9
:104C00000022B64B02F0F8FC002200230E900F9118
:104C100001F002FF002800D14CE100230022200017
:104C2000290001F0F9FE0222431E9841131AAC4AF2
:104C30003900019202220AA80092524600F09EFA20
:104C40004B46002B13DA8022120694467B684042C2
:104C500063447B60FB686344FB6008E002000B0078
:104C60003A607B60002200230020BA60FB6010B035
:104C70001CBC90469946A246F0BD02000B0002F013
:104C800035FFB860F960386079600020EFE7D32223
:104C90008E4B520502F02AFF924A934B04000D00FE
:104CA00002F024FF02000B0020003A607B60290024
:104CB00002F01CFF8B4A8C4B02F018FFB860F960C1
:104CC0000120D4E700F056FF884A894B04000D000C
:104CD00002F092FC0022874B02F054F803F05AFADB
:104CE000804603F08DFA764A764B0690079102F0E3
:104CF00083FC02000B002000290002F0F7FE734B3A
:104D000002900391069807996F4A02F075FC43469A
:104D100004000D00049405951F2B30DC013B764AFE
:104D20009B009B589E422AD002000B0002980399D8
:104D300002F0DCFE02000B0005000C003A607B6014
:104D4000029803992A00230002F0D0FE049A059BE2
:104D500002F0CCFE06000B003200BA60FB604B464E
:104D60004046002B00DB82E780231B069C46644400
:104D700061443D607C60BE60F960404277E7049A20
:104D8000059B0298039902F0B1FE0B0002003A6005
:104D90007B604B0036155B0D05000C00F31A102BE1
:104DA000CEDD06980799D322484B520502F024FC29
:104DB00004000D0002000B000298039902F096FE19
:104DC00002000B00029803990892099302F08EFEEC
:104DD00022002B0002F08AFE04000D0006980799BD
:104DE000404A414B02F008FC22002B0002F07EFEFC
:104DF00002000B00049005910898099902F076FED4
:104E000002000B003A607B604B005B0DF61A050058
:104E1000089A099B0C0002920393312E90DD0698AC
:104E20000799B822304B920502F0E6FB04000D0012
:104E300002000B000298039902F058FE0A000100DC
:104E400013000291039202000898099902F04EFEA5
:104E500022002B0002F04AFE04000D00069807997C
:104E6000264A274B02F0C8FB22002B0002F03EFE30
:104E700002000B000492059358E7124B01F082FFE9
:104E8000104B04000D009E423CD00F4A0F4B01F026
:104E900079FF02000B0020003A607B60290002F0DD
:104EA00025FE094A094B01F06DFFB860F960012049
:104EB0004042DCE60323BAE6FB21E93F7BD902400E
:104EC00000004054FB21F93F3163621A61B4D03DC8
:104ED000FB213941FFFFEF7FEAFBFFFF000070413C
:104EE00064A600007370032E8A19A33B83C8C96DA2
:104EF000305FE43F0000E03FE4A50000C149202509
:104F00009A837B39D3220D4B520501F03BFF0C4AAB
:104F10000C4B04000D0001F035FF02000B002000D7
:104F20003A607B60290002F0E1FD054A054B01F083
:104F300029FFB860F9600120404298E661B4D03D95
:104F40007370032E8A19A33BF0B54F464646C0B492
:104F500087B000920193754B4F00814688467F08C9
:104F60009F4263DC03F016F9002800D1DAE04A46DC
:104F700043464846414602F03FFB04000D006C4AA0
:104F80006C4B02F039FB6C4A6C4B01F0FBFE2200CB
:104F90002B0002F031FB6A4A6A4B02F0A7FD2200A7
:104FA0002B0002F029FB684A684B01F0EBFE22005F
:104FB0002B0002F021FB664A664B02F097FD2200AF
:104FC0002B0002F019FB644A644B01F0DBFE220067
:104FD0002B0002F011FB029003910022604B200095
:104FE000290002F009FB029A039B06000F00200033
:104FF000290002F001FB009A019B04000D004846C5
:10500000414602F0F9FA02000B002000290002F0EC
:105010006DFD02000B003000390002F067FD020058
:105020000B0000204F4902F061FD70E002000B0010
:1050300002F0E2FA04000D003D4A3E4B02F0DCFAB9
:105040003D4A3E4B01F09EFE22002B0002F0D4FAB6
:105050003B4A3C4B02F04AFD22002B0002F0CCFA06
:10506000394A3A4B01F08EFE22002B0002F0C4FABE
:10507000374A384B02F03AFD22002B0002F0BCFA0E
:10508000354A364B01F07EFE2B00220002F0B4FAC6
:10509000354B029003919F429FDD344B00229F428B
:1050A0003ADC334900207B182E4916001F0002F01D
:1050B0001DFD049005910022294B2000290002F0DB
:1050C0009BFA32003B0002F011FD029A039B06009E
:1050D0000F002000290002F08FFA009A019B0400C3
:1050E0000D004846414602F087FA02000B002000FE
:1050F000290002F0FBFC02000B003000390002F036
:10510000F5FC02000B000498059902F0EFFC07B0D3
:105110000CBC90469946F0BD164B002604920593B0
:10512000154FC8E700200F49F1E7C046FFFF3F3E9B
:10513000D43888BEE9FAA8BDC4B1B4BD9EEE213E04
:10514000AD529C804F7E923E9015CB19A001FA3E45
:105150007751C1166CC1563F4C5555555555A53F15
:105160000000E03F0000F03F3233D33F0000E93F52
:105170000000E0FF0000E73F0000D23FF0B55646D8
:105180004D4644465F46F0B48E4CA5440991190043
:105190001400A89A0B938C4B9200D2580B000290EB
:1051A000013BE01E18211D0016000892009301F03B
:1051B00029FBC3430200DB171A401300110001331F
:1051C0000E929A009B1ADB001B1906934C1B761952
:1051D00018D4A99BA5009C46361926AF6544013614
:1051E00007E0286803F00CF8013403C70435B44223
:1051F00008D0002CF5DA00200021013403C7043563
:10520000B442F6D1089B002B01DA00F0F9FB76AB33
:1052100019008B4626AA9146089A0A930132D200B9
:105220009344029A9A469046009BDB0099440833C7
:105230009844009B002B00DAB5E14C46002600277D
:10524000029D2268636803CD02F0D6F902000B00CC
:105250003000390001F096FD083C06000F0045457E
:10526000EFD15346C0C39A4608239C46E144DA4531
:10527000DFD10899554A0B00944663449B0012A85D
:1052800084461A000298624483460D920B9A0433B6
:10529000D200634493440F930591059A0A98D30072
:1052A00019000C938C46030063441E685F68002A53
:1052B00034DD12AB99461300454A80469446634458
:1052C000DB00984474AB9A460022424B3000390010
:1052D00002F092F902F05EFF02F092FF00223E4BD4
:1052E00004000D0002F088F902000B0030003900C4
:1052F00002F0FCFB02F04EFF4B4601C399464346C9
:1053000020001A685B68290001F03CFD08235B421D
:105310009C46E04406000F00D045D5D1069B3000E6
:105320001A003900994600F0C1FCFF2300229B05BA
:1053300004000D0002F060F900F020FC0022274B71
:1053400002F05AF902000B002000290002F0CEFB07
:1053500004000D0002F01EFF804602F051FF020023
:105360000B002000290002F0C1FB4C4606000F0094
:10537000002C00DCF8E0059B18205A1E920012ABAE
:105380009B58001B19000141884481405B1A12A9F7
:105390008B501722121B13410793079B002B4BDDE9
:1053A00001239C46059BE044002B00DCF2E28025B3
:1053B0001096119712AB0021002409486D04059F37
:1053C00019E0C04684FDFFFF6CA70000FEFFFF3F11
:1053D000FFFFFF1F0000703E0000704100002040F2
:1053E000FFFFFF00002A02D0AA1A1A60013401311F
:1053F00004338F4209DD1A68002CF3D0821A013180
:105400001A60012404338F42F5DC109E119F069B25
:10541000002B0EDD012B00D1B1E0022B09D1059B41
:1054200012A95A1E920012AB9B5810939B029B0A22
:105430008B50079B022B7ED00023002230003900C6
:1054400001F0EAFA059B002800D16BE208995A1E88
:10545000914210DCBF490F988C4612A963448C46D8
:1054600000219B0063441C68043B21438342FAD122
:10547000002900D0B5E0089B12AA013B9B00D3583D
:10548000002B00D084E201220D9B043B59680132BD
:105490000029FAD005990B008C460133624407922B
:1054A000934242DC0E9A9446A99A634492460B9A20
:1054B0009B00944626AA90469A44059B0A9A634408
:1054C000DB0098440C9B94469946079BE144DB0023
:1054D000634405935346186802F092FE43461860F1
:1054E0005960009B002B23DB444600260027029DC9
:1054F0002268636803CD02F07FF802000B003000E1
:10550000390001F03FFC083C06000F005D45EFD17B
:105510004B469E60DF6004239C460433E2449C4675
:10552000059BE144E0449945D4D1079B0593B4E63B
:1055300000260027ECE732003B000020864902F0FD
:10554000D5FA06000F00002C00D175E7069A00205E
:10555000814900F0ABFB02000B003000390002F083
:10556000C5FA06000F0067E7069B002B12D1059BCA
:1055700012AA013B9B00D558EB1507930DE7059B3D
:1055800012A95A1E920012AB9B5810935B025B0A41
:105590008B504EE70022714B01F062FA00280ED1C9
:1055A0000023079348E7534600260027C0C39A46C6
:1055B00008239C46E144DA4500D03AE659E6012347
:1055C0009C4601330793059BE044002B00DDEEE68B
:1055D00032003B000020604902F088FA06000F000C
:1055E0002AE743460B93069B12A8183B1900069323
:1055F0009300C3580092002B0FD1564813008446E5
:1056000012A8634484469B006344043B5868013AF3
:1056100018390028F9D000920691069A00204E49C8
:1056200000F044FB009B04000D00002B00DAB3E106
:1056300012AA94469F00DB0067449C460A9A059391
:10564000624493461600386802F0DAFD22002B000F
:1056500001F0D2FF424B306071600022200029002F
:1056600001F0CAFF083E74AB04000D00043FB342D2
:10567000E9D100239A464EAB0293089B99464B46CC
:1056800000260027002B21DB8020364B5D46984604
:10569000C005354900260027002408E008239C4661
:1056A0000835E044A24511DB4346186859682A686A
:1056B0006B6801F0A1FF02000B003000390001F01F
:1056C00061FB013406000F00A145E7DA029A534658
:1056D0009446DB0063441E605F6001239C46093BE7
:1056E000E2449C4674ABE3449B45C8D1029B994677
:1056F000A89B022B00DD82E0002B37DC1DD1059B2F
:1057000000254B441E0000243268736828002100E5
:1057100001F038FB009B05000C00083E5A1E009269
:10572000F2D2079B002B03D080231B069C466444C7
:105730002A00230009990A604B6007200B9B184040
:105740009F239B009D443CBC90469946A246AB4695
:10575000F0BDC046FFFFFF3F0000F03F0000E03F0C
:105760000000703E80A70000FB21F93F059B002050
:105770004B441E0000214CAF32687368083E01F0B4
:1057800001FBBE42F8D1079B002B24D08023099A4D
:105790001B06CB18106053600B0002004E984F9907
:1057A00002F0A4F9009B002B0BDD012450AD0CCDC1
:1057B00001F0E8FA009B0134A342F8DA079B002BC2
:1057C00003D080231B069C4661440B00020009990C
:1057D0008A60CB60B1E702000B00099C2260636025
:1057E0000B0002004E984F9902F080F9009B002BAD
:1057F000DBDC0B00020009998A60CB609DE7A89B67
:10580000032B9AD1009B002B00DCE3E07E4A059B32
:1058100094464B441E685F68009B63449A46DB00D5
:105820004B4498464CAB9B4643465C681B6818004B
:10583000210032003B000290039101F0A3FA040022
:105840000D0002000B000298039902F04FF93B0093
:10585000320001F097FA43469860D9601C605D60A1
:1058600008235B429C46E04426002F00C345DBD161
:10587000009B012B00DCADE0059BC8464B441E6835
:105880005F685346DB009B46D844434630005C6863
:105890001B683900009301941A00230001F072FA8A
:1058A00004000D0002000B000098019902F01EF99F
:1058B0003B00320001F066FA43469860D9601C60F4
:1058C0005D6008235B429C46E04426002F00C145F2
:1058D000DBD15D460027002408354D4450AE2A68D0
:1058E0006B683800210001F04DFA083D07000C00FC
:1058F000AE42F4D1079B002B71D0099A4E994B46CA
:105900001160802109068C465B68494663445360F8
:105910004B46DB688968634464449160D3601761D7
:1059200054610AE7994643460B93069B30005A425E
:10593000390000F0BBF90022344B04000D0001F0E7
:105940008FF8002832D0324B00222000290001F0CD
:1059500053FE02F01FFC4A460600970002F050FC7E
:1059600000222A4B01F048FE02000B002000290013
:1059700002F0BCF802F00EFC12AAD0514A46069B77
:105980000132183300920693930012AAD65044E6CF
:1059900001227FE500243AE5A89B022B14DC002BB2
:1059A0000FDC00D0C9E600250024BAE64B462000F3
:1059B00029009E0002F0EEFB12AB98514B4600937B
:1059C0002BE600200021DEE64EAB9946A89B032B78
:1059D00000D0B2E6079B00270024002B8DD14E9A01
:1059E0004F9B09990A604B604B469A68DB680092AE
:1059F00001938A60CB603A0023000A614B619CE608
:105A000076AB0A9335E4C046FFFFFF1F00007041EC
:105A10000000703EF0B54F464646C0B487B00092D5
:105A20000193464A4B00814688465B08934205DC59
:105A300002F0B0FB4146031E484666D04A46434644
:105A40004846414601F0D8FD04000D0002000B005D
:105A50004846414601F0D0FD394A3A4B06000F0056
:105A60002000290001F0C8FD374A384B02F03EF80B
:105A700022002B0001F0C0FD354A364B01F082F9BF
:105A800022002B0001F0B8FD334A344B02F02EF80F
:105A900022002B0001F0B0FD314B324A01F072F9C7
:105AA0000E9B02900391002B34D0009801990022A4
:105AB0002D4B01F0A1FD029A039B0490059130004B
:105AC000390001F099FD02000B000498059902F0DD
:105AD0000DF822002B0001F08FFD009A019B02F0CF
:105AE00005F8224A04000D00214B3000390001F076
:105AF00083FD02000B002000290001F043F90200A1
:105B00000B004846414601F0F1FF07B00CBC90463F
:105B10009946F0BD02000B002000290001F06CFD49
:105B2000124A134B01F0E2FF32003B0001F064FD2A
:105B30004A46434601F026F9E7E7C046FFFF3F3EED
:105B40007CD5CF5A3AD9E53DEB9C2B8AE6E55A3E07
:105B50007DFEB157E31DC73ED561C119A0012A3FA3
:105B60001111813FA6F810110000E03F495555552D
:105B70005555C53F49004B0819007047454AF8B5CF
:105B8000564692464B005B0D9A444D465F4644464E
:105B90005246F0B4894605000C000E000700132A97
:105BA00022DC002A47DB52463B4B134198460B0050
:105BB00042461340034311D0384A394B01F0E2F812
:105BC0000022002300F042FF002805D0002C41DB1A
:105BD0004E46434600279E43380031003CBC904669
:105BE0009946A246AB46F8BD5246332A08DD8023CB
:105BF000DB009A45F2D102000B0001F0C3F8EDE79B
:105C0000284A9446012263445242DA4093460242B3
:105C1000E4D0224A224B01F0B5F80022002300F024
:105C200015FF0028D8D0002C1ADB5B464E469F4358
:105C300038003100D2E7194A194B01F0A3F80022CD
:105C4000002300F003FF0028C6D0002C16DB00273D
:105C50000026C1E7802352465B0313419944B7E70E
:105C60005346142B12D03423524601279B1A9F40CF
:105C70007F19AF429B415B429944D6E764006408B8
:105C800025430027002DA7D0074EA5E7133B9C46D0
:105C9000E144CAE701FCFFFFFFFF0F009C7500888D
:105CA0003CE4377EEDFBFFFF0000F0BF4B0070B51A
:105CB0005B0D14000A00002B1AD14B005B08034354
:105CC00015D00022224B01F097FC224B0A009C4287
:105CD00022DB4B005B0D363B1F4DE318AB4220DC53
:105CE000002B0DDD1D4C1B0522401A43110070BD19
:105CF0001B4DAB42F0D102000B0001F043F8F6E778
:105D00001D00353518DA174B02009C420ADC0B00E7
:105D10001548164900F032F8134A144B01F06CFC98
:105D2000E5E702000B001248124900F027F8104A7C
:105D3000104B01F061FCDAE7084C363322401B05BA
:105D40001343190000220C4B01F056FCCFE7C0466C
:105D500000005043B03CFFFFFE070000FFFF0F8034
:105D6000FF07000050C3000059F3F8C21F6EA501E1
:105D70009C7500883CE4377E0000903C30B54A00BA
:105D8000DB0FDB0752081A43110030BDF7B50600E0
:105D90000D000C008B180193019B671B9C4207D0E0
:105DA000336821781B683000984701340028F3D10C
:105DB0003800FEBD70B505000C00081E07D002F0CB
:105DC00089FF2B6802005B6821002800984770BD9E
:105DD00010B5FFF7EFFF10BD10B540220021040001
:105DE00002F04BFB002320002364636410BD3F23BB
:105DF000026C10B5541C2340446C9C4201D0815469
:105E0000036410BD0023036443647047436C026C59
:105E1000934206D03F21C25C01330B404364100023
:105E200001E0012040427047036C406C181A00D515
:105E300040307047436C026C934201D0C05C01E07B
:105E4000012040427047036C406C5A1C3F231340B2
:105E5000181A42424241D0B27047000003210A485A
:105E600002680A430260094802680A43026008495E
:105E7000084A094B9B1A03DD043BC858D050FBDC91
:105E800000F012F8FAF776F92405004054050040B6
:105E900054AA000000000020A0020020FEE7FEE758
:105EA000FEE7FEE7FEE7FEE72D4B10B51A78012A64
:105EB00019D12C4A1268120715D12B4AE024116817
:105EC000F0220800104021420BD1284909681142F4
:105ED00009D12749274A11608021274A0902116008
:105EE00001E03028F1D01A78012A0DD11D49096846
:105EF000090709D1F0201C4909680140402903D154
:105F00001A490968014223D01B68DBB2012B25D155
:105F1000144B1B681B0721D1134B1A68F0231A403E
:105F2000A02A04D1114A12681A4203D016E0D02ADE
:105F300014D1F7E7114B1A68012A03D1C022104B84
:105F40001A600BE00F4A1A601A68012AFCD1F5E7C3
:105F5000C1218020C900C0054250D5E710BDC04610
:105F6000E00F00F0E40F00F0E80F00F0EC0F00F09D
:105F7000DFFF07C004050040186C004000EC06403D
:105F800014EC0640759300000120704710B50368BB
:105F90001322DB69984710BD704700000369054A6A
:105FA0009950FC331A6A002AFCD0002201201A62A0
:105FB0007047C0461C050000030010B55C331A781A
:105FC0001F2313400122110099400D4B0424D9676F
:105FD000C221036989005C505A60DA60A022002166
:105FE000D20099500122074952425A5006491430B2
:105FF0005A500C395A5008315A50FFF703FF10BD60
:1060000004E100E00C0500001405000010B5143098
:10601000FFF70AFF10BD10B51430FFF70BFF10BDDE
:1060200010B51430FFF7F2FE10BD0000030070B58C
:106030005E331C780269604BD45003005D331C78DA
:106040005E4BD450030061331C785D4B012C0CD1A6
:1060500005005F352E78A225ED005651050060350C
:106060002E78A125ED00565100E00024D45096234F
:10607000DB00994238D996231B01994237D99623E0
:106080005B01994236D996239B01994234D9E12389
:106090009B01994232D99623DB01994231D9E12300
:1060A000DB0199422FD996231B0299422DD9E12376
:1060B0001B0299422BD996235B02994229D9E123ED
:1060C0005B02994227D9E1239B02994225D93D4B96
:1060D000994224D9E123DB02994223D9E1231B030E
:1060E000994221D8384B21E09E23DB021EE09D23FC
:1060F0001B031BE0354B19E0354B17E0EC239B03EA
:1061000014E0344B12E0344B10E0344B0EE0344BCF
:106110000CE0344B0AE0344B08E0344B06E08023BB
:10612000DB0403E0324B01E080235B0531490024AE
:1061300053500423243953501100FC31CC600C62BD
:10614000C1210134890014605C309460535003789D
:106150001F202200D9B20840824080342648FF34F4
:106160005BB20251002B13DA0F230B40083B234C88
:106170009B089B001B1903242140A140FC348C4048
:10618000DD69A543C0248C4021002943D96111E079
:10619000194C9B089B001B1903242140A140C025DA
:1061A000FC348C40AD005E59A643C0248C402100D5
:1061B00031435951026070BD0C0500001405000008
:1061C0006C05000090D0030000D0BE0E00B013009C
:1061D0000050270000A04E0000F0750000509D0008
:1061E00000F0EB0000903A0100E0D70100B0AF03EF
:1061F00000705F072405000000E100E000ED00E012
:10620000F7B5009308AB1B7800250193FA2304002F
:106210009B0083600E4B45600833036014300F0011
:106220001600FFF7D9FD23005C3327611E70009B29
:10623000084A9B00995823005D331970019B200088
:106240009B009A5823005E33DD701A70FEBDC04675
:10625000C0A7000068A50000036910B51A00FC3251
:10626000D2680400002A0AD0A322D2009958143020
:10627000C9B2FFF7BCFD00222369FC33DA6010BD10
:1062800010B50248FFF7E8FF10BDC04668110020B6
:106290001D2307B502220093024901330248FFF78C
:1062A000AFFF07BD002000406811002070470000CC
:1062B00010B500F011F8FFF7F9FF012000F0F0F938
:1062C000FEF7A2F9FEF7B4F9024B002BFAD000E07A
:1062D00000BFF7E700000000C421114A89005058B0
:1062E000104B0340C02000020343535080239139D8
:1062F0009B02FF39535013608023A3220021DB054A
:10630000D20099500122A1209A60074BC000195079
:10631000C120023180001950403019501A60704776
:1063200000E100E0FF00FFFF00100140014B18609A
:106330007047C046DC010020F7B500231E2877D83F
:106340003C4B8000C258042A14D006D8022A0DD033
:106350000ED80423012A14D069E0062A0ED00BD3EC
:106360001A2A0DD002231B2A0BD060E0082308E074
:10637000102306E0202304E0402302E0802300E015
:1063800001232D4A1268082A04D9092A05D00A21B6
:10639000022404E00821002401E011000124A025CA
:1063A00001261C272548ED004651254D254E2D6818
:1063B0001B02AD003D400195234D2D680095855988
:1063C000AC466746214D3D401D4385518359C0254C
:1063D0009C46009BAD021D40FF2367461B023B40CD
:1063E0002B43019D1D43009B5F0160231F402B0039
:1063F0003B431C4301238451154C036063680F48E1
:10640000002BFBD00024124B01255C60A123DB0094
:10641000C3584560A025ED0044511BB2914207D0FE
:1064200002D98A1AD34003E0521A934000E00023B5
:106430001800FEBD68A50000E001002000700040CB
:10644000D801002004050000D4010020FF00FFFF58
:10645000FC700040F0B51E286CD8374B8000C25845
:10646000364B1E68002E2ED1C2243548A400075991
:10647000344B03253B40C0273F023B43035180235D
:10648000893C9B00FF3C03512F4F03602F4B803C06
:10649000D859FF3CA043D8510437D859A8432043CA
:1064A000D8510837D8590C35A843083D2843D8514E
:1064B000A820C0001E508026C120760280001E50F9
:1064C0001C601E4B1C6000231426214834005C43D2
:1064D000255804006F1C0FD1142058432250A020CF
:1064E0000325C132FF329200C0051550194A080039
:1064F0001268082A03D10BE0AA4218D1ECE7082A57
:1065000002D9083AD14002E00820821A91400800DE
:1065100014225343E3189A680C495132FF32920017
:1065200058605050DA68C1239B00CA5002E0013322
:10653000032BCBD1F0BDC04668A50000CC110020D4
:1065400000E100E0FF00FFFF0405000000900040B4
:10655000E4010020DC0100201E4BF0B5596C18004E
:106560001D4A002914D0A025A12600230124ED05F1
:10657000F600D1584F1C06D0D7187F68002F02D0E4
:1065800027008F40AF5114333C2BF2D100234364DA
:10659000131DA02540329446002001240F4EED0526
:1065A000DA680F49920057180A495218526C002AAB
:1065B0000CD01A1F1268511C05D01968FF2902D08F
:1065C00021009140A9513A00FC32506414339C459B
:1065D000E6D1F0BDFC900040E40100200C05000075
:1065E0000090004000B51E2816D80C4A83009B5826
:1065F000032911D8A0220800C133FF33D2059B0024
:1066000000F06CF802080406002104E00C2102E00E
:10661000042100E00321D15000BDC04668A5000060
:106620001E280DD8074B8000C058A0220123D20598
:106630008340002901D1044901E0A121C900535040
:106640007047C04668A500000C050000030000204C
:106650001E2B0AD8A222A021D200C9058858034ABD
:106660009B009B58D84001231840704768A5000044
:10667000084A0949094B10B51B688858FA22190ABB
:106680001B0618439200002300F0F4F94904C00BE4
:10669000084310BD0405000000100140D011002087
:1066A00070B5041E09D0FFF7E3FF050000F014F8F1
:1066B000FFF7DEFF401B8442F8D870BD0022044B78
:1066C0009A60044A13680133DBB213607047C04616
:1066D000FC100140D01100207047000002B4714648
:1066E00049084900095C49008E4402BC7047C04615
:1066F000002243088B4274D303098B425FD3030A01
:106700008B4244D3030B8B4228D3030C8B420DD313
:10671000FF22090212BA030C8B4202D312120902A1
:1067200065D0030B8B4219D300E0090AC30B8B42DF
:1067300001D3CB03C01A5241830B8B4201D38B038D
:10674000C01A5241430B8B4201D34B03C01A524132
:10675000030B8B4201D30B03C01A5241C30A8B4275
:1067600001D3CB02C01A5241830A8B4201D38B0260
:10677000C01A5241430A8B4201D34B02C01A524104
:10678000030A8B4201D30B02C01A5241CDD2C30976
:106790008B4201D3CB01C01A524183098B4201D3F2
:1067A0008B01C01A524143098B4201D34B01C01ADD
:1067B000524103098B4201D30B01C01A5241C30855
:1067C0008B4201D3CB00C01A524183088B4201D3C4
:1067D0008B00C01A524143088B4201D34B00C01AB0
:1067E0005241411A00D20146524110467047FFE71C
:1067F00001B5002000F0F0F802BDC0460029F7D036
:1068000076E7704703460B437FD4002243088B4250
:1068100074D303098B425FD3030A8B4244D3030B27
:106820008B4228D3030C8B420DD3FF22090212BAEC
:10683000030C8B4202D31212090265D0030B8B4268
:1068400019D300E0090AC30B8B4201D3CB03C01A52
:106850005241830B8B4201D38B03C01A5241430B2D
:106860008B4201D34B03C01A5241030B8B4201D31D
:106870000B03C01A5241C30A8B4201D3CB02C01A88
:106880005241830A8B4201D38B02C01A5241430A00
:106890008B4201D34B02C01A5241030A8B4201D3EF
:1068A0000B02C01A5241CDD2C3098B4201D3CB0196
:1068B000C01A524183098B4201D38B01C01A524145
:1068C00043098B4201D34B01C01A524103098B4249
:1068D00001D30B01C01A5241C3088B4201D3CB0034
:1068E000C01A524183088B4201D38B00C01A524117
:1068F00043088B4201D34B00C01A5241411A00D2C7
:1069000001465241104670475DE0CA0F00D049422F
:10691000031000D34042534000229C4603098B429F
:106920002DD3030A8B4212D3FC22890112BA030A27
:106930008B420CD3890192118B4208D389019211A9
:106940008B4204D389013AD0921100E08909C3092E
:106950008B4201D3CB01C01A524183098B4201D330
:106960008B01C01A524143098B4201D34B01C01A1B
:10697000524103098B4201D30B01C01A5241C30893
:106980008B4201D3CB00C01A524183088B4201D302
:106990008B00C01A5241D9D243088B4201D34B001D
:1069A000C01A5241411A00D20146634652415B105F
:1069B000104601D34042002B00D549427047634640
:1069C0005B1000D3404201B5002000F005F802BD85
:1069D0000029F8D016E770477047C046D0400B1C1E
:1069E0001141203A03D49C46134118436346524256
:1069F000934018437047C0468446101C62468C463C
:106A0000191C634600E0C0461FB500F08BFD00284E
:106A100001D40021C8421FBD10B500F0DFFC404288
:106A2000013010BD10B500F07DFD002801DB002015
:106A300010BD012010BDC04610B500F073FD002848
:106A400001DD002010BD012010BDC04610B500F0D2
:106A500005FD002801DC002010BD012010BDC0464E
:106A600010B500F0FBFC002801DA002010BD012069
:106A700010BDC046F0B54F464646C0B41604360CAD
:106A80009946330005042C0C070C150C63437E4318
:106A90006F4365431C0CAD1964199C46A64203D98B
:106AA00080235B02984647446346250CEF191D047A
:106AB0004B464A4343432D0C240464199918C919C1
:106AC00020000CBC90469946F0BDC046F0B5574634
:106AD0004E4645464300E0B446028846760A1F0EFD
:106AE000C40F002F47D0FF2F25D0002380259A46C2
:106AF0009946F600ED042E437F3F434642465D0231
:106B0000D20F5B006D0A1B0E904640D0FF2B39D090
:106B100080220020ED00D20415437F3BFB18424643
:106B20005746591C62408C4607430F2F5CD86F496B
:106B3000BF00C9598F46002E45D108239A46063B0F
:106B40009946DAE7424602282DD0032800D1C3E057
:106B5000012800D0A2E0002500260240D4B276022F
:106B6000ED05760A2E43E407264330001CBC904610
:106B70009946A246F0BD002E1AD104239A46033B43
:106B80009946BAE72A00511E8A41901CC6E70120A7
:106B9000002DC3D0280001F0C9FB431F76309D4073
:106BA00043420020BAE70124FF2514400026D6E71F
:106BB000300001F0BBFB431F9E400023763047426C
:106BC0009A46994699E70C239A46093B994694E7D9
:106BD00080260024F603FF25C1E735004846B2E7CA
:106BE000350022004846AEE72904090C0800370C9E
:106BF0003604360C2C0C7943704367437443060CFF
:106C000064183619B14203D98021490288464744A5
:106C10000004000C310409188D01681E8541890E9D
:106C20002943350CED19AD010D43290104D501238C
:106C300069081D4063460D4319007F31002925DD99
:106C4000680704D00F202840042800D0043528010C
:106C500003D5274980330D401900FE29A3DC012408
:106C6000AD016E0A1440CDB279E78020C003064220
:106C700007D0054205D128434602760A4446FF253F
:106C80006DE706437602760AFF2568E70124611A5C
:106C90001B2905DD14400025002660E76346CBE78D
:106CA0002E002023CE40591A8D406B1E9D412E434D
:106CB000730704D00F233340042B00D00436730134
:106CC00004D5012401251440002648E70124B6011B
:106CD000760A1440002542E780260124F6032E435D
:106CE0007602760A1440FF2539E7C046F0A7000077
:106CF000FFFFFFF770B5002830D0C317C5185D40FF
:106D0000C40F280001F012FB9E231B1A962B0DDCEA
:106D10009622D21A95406A02520AD8B25202C0058F
:106D2000520AE40702432243100070BD992B19DC7C
:106D30009922D21A9540124A2A40690704D00F219D
:106D40000D40042D00D00432510103D50C4B1A40E4
:106D50009F231B1A9201520AD8B2DFE700240020B9
:106D60000022DBE705222E00121AB921D6402A00A4
:106D7000C91A8A40551EAA4135001543DBE7C046B3
:106D8000FFFFFFFBF8B556465F464D464446F0B45C
:106D90000F00FD0FAA4609037C002E005F00450F7F
:106DA000490A7F0D2943C5001803BC46400A570F06
:106DB000640DDB0F3843D2009A4500D1AAE0664645
:106DC000A61B002E00DCFFE06346002B39D1030038
:106DD000134300D0D9E06B0709D00F232B40042BBD
:106DE00005D02B1DAB42AD416D4249191D000B0270
:106DF00000D482E0CA4B01349C4200D1FEE00A007C
:106E00005646C84BED081A40500764055202054328
:106E1000120B640D002112030B0D1B056405120BF0
:106E20001A436308C04CF60714401C43640064080E
:106E30003443280021003CBC90469946A246AB460C
:106E4000F8BDB74B9C42C6D080231B041843382E94
:106E500000DDEBE01F2E00DD1EE120239B1B9C4686
:106E600003006746BB40984613004746F3403B4348
:106E70006746BA40571EBA4113430200F240EB1A6C
:106E80009D42B6411D008A1A7642911B0B0231D5F4
:106E90004A02560A002E00D1B4E0300001F046FA52
:106EA0000300083B1F2B00DDB5E020222900D21A89
:106EB000D1409E400A009D4032439C4200DDB1E03B
:106EC0001C1B631C1F2B00DDD5E0202114002800B3
:106ED000C91A8C40D8408D400443DA40681E854171
:106EE00011002543002476E74146314300D134E2C6
:106EF000310045466B0700D06FE756464807ED085E
:106F0000C9080543864B9C4235D00A036405120B21
:106F1000640D7FE76346E31A9B46002B00DC8BE0A1
:106F20006746002F3CD07E4FBC4200D153E78027FC
:106F30003F0438435B46382B00DCF7E00243501E29
:106F400082410020D2B253194218AB4289411D0040
:106F5000494289180B02CDD5714B01349C4200D1B6
:106F60003DE101206F4A6B080A4028401843D507CD
:106F7000054351082FE72B000B4300D1CBE18023C1
:106F80001B030B431A03120B44E7013E002E6DD185
:106F9000AE1AB5429B41091A5B42C91A350075E722
:106FA0000700174300D116E701235B429C46E344E8
:106FB0005B46002B00D0E0E0AA18AA429B410918CA
:106FC0005B4259181500C5E7002E75D1661C760581
:106FD000760D012E00DCF3E0AE1AB0464545BF4108
:106FE0000E1A7F42F61B370200D48FE0551BAA42CF
:106FF000B641411A76428E1B9A464BE7564600220E
:10700000002507E7280001F091F920300300083B34
:107010001F2B00DC49E72A002838824000259C42CB
:1070200000DC4DE73F49E41A1140D4E60243501E0C
:107030008241D3B2002222E7002B00D0F3E0631C90
:107040009C465B055B0D012B00DC9FE0344B9C45AF
:1070500000D1C3E0AA180918AA4280414042411851
:10706000CD075208154349086446B4E62C4B9C42B0
:1070700000D0ECE6AFE611001F3CE1400C00202BF5
:1070800000D17FE04021CB1A9A4015436A1E9541FA
:107090000021254300242DE733000700203BDF407B
:1070A0003B00202E70D04027BE1BB0400243501E34
:1070B000824113430022E2E6002C4FD0184CA44535
:1070C00000D1ABE08024240476422143382E00DD39
:1070D000DFE01F2E00DD43E12027BC1BA1460C0092
:1070E0004F46BC40A0462C004746F4403C434F4628
:1070F000BD406F1EBD41F1402C43151BAA42924179
:10710000411A5242891A64469A46BFE641464546AC
:10711000314300D0BEE6002600240025F2E6C0463A
:10712000FF070000FFFF7FFFFFFF0F801F2B59DCD1
:107130002027FF1ABC46070063469F405B46B946BE
:107140001700DF40B8464F4643461F4363469A4008
:10715000531E9A415B463A43D840F4E60C002C4358
:107160005CD0F643002E55D1551BAA42A441411ACA
:107170006442091B9A46644688E6964FBC4200D09A
:10718000D8E628E6002280E700208FE70B002B439B
:10719000002C00D0C2E0002B00D101E1030013431A
:1071A00000D118E6AB18AB42B64109187642711807
:1071B0000A0200D409E1884A1D00114064460AE62B
:1071C000002C5BD10E002E4300D08AE00100114359
:1071D00000D1C2E0010015009A46FCE5644600219A
:1071E00000258FE620235B429C46DC446346070073
:1071F000DF405B46BC46202B00D1ACE040235F461D
:10720000DB1B98400243501E8241634613431A0021
:10721000002098E66F4CA44500D057E70100150008
:1072200064469A46D7E5002C39D10C002C436ED029
:10723000DB43002B1AD0674CA44568D0382B00DD07
:10724000A4E01F2B00DDAEE020240F00E41AA740CD
:10725000B9462F00DF40B846A3464F464446274371
:107260005C46A5406C1EA541D9403D43AD189542F2
:107270009B4109185B42591864466BE60C002C438D
:1072800015D1010011437BD0010015009A46514CE5
:10729000A1E50D43691E8D410021ECB22DE74D4C57
:1072A000A44534D0802424045B422143C6E7040073
:1072B00014434ED0ED084C072C438025C9082D03FC
:1072C000294208D0C6082E4205D1D20841071143F1
:1072D0000C009A463100620FC900E50011433D4C95
:1072E00079E50600164300D175E5AE1AB04645456E
:1072F000BF410E1A7F42F61B370200D4F4E5551B3E
:10730000AA42B641411A7642891B9A4663E50100BA
:10731000150064465FE5002200257BE5002B3BD08D
:107320000300134315D0ED084B072B438025C908F4
:107330002D03294207D0C4082C4204D141070B0079
:107340002100D2081343C9005A0F1143DD00214C1C
:1073500041E5204C3FE5002054E700260025D1E51B
:1073600034000F00203CE7403C00202E2BD040276B
:10737000BE1BB1400D43691E8D4100212C43BCE66C
:10738000802100260903134C0025BBE50D43691E2F
:107390008D410021EDB269E7010015000D4C1AE5A1
:1073A0000100150017E51C000F00203CE7403C00E1
:1073B000202B0CD04027FB1A99400D43691E8D41AC
:1073C0000021254352E70021D4E71D0092E500216A
:1073D000F3E7C046FF070000FFFF7FFFF0B55F4601
:1073E00056464D464446F0B41F035C00DB0F9A46F8
:1073F000194B0E034D00C90F8046360B6D0D8B46A1
:1074000091463F0B640D9D4219D0134B9C421BD0FB
:107410000123A54206D018003CBC90469946A246DE
:10742000AB46F0BDBE42F6D1C845F4D1D34510D02D
:10743000002DF0D1304303005A1E9341EBE7310099
:1074400001230143E7D1E0E73A430123002AE2D1D7
:10745000DEE70023DFE7C046FF070000F0B55F4628
:10746000444656464D46F0B41F033C0B2C4F0E03CA
:107470004D00A3465C008446360B6D0DC90F904647
:10748000640DDB0FBD422BD0254FBC422ED0002D0A
:107490000ED130430700814678427841002C17D145
:1074A0005F463A4314D14B460020002B0AD006E039
:1074B000002C02D15846024301D099421AD0012330
:1074C000484218433CBC90469946A246AB46F0BDA4
:1074D0000028F2D058425841012240421043F1E7BF
:1074E00037000743D0D002204042EBE75F46174306
:1074F000CDD0F8E7A542E2DC05DB5E45DFD808D059
:1075000000205E45DED248424841012340421843F4
:10751000D8E7C445D3D80020C445F4D3D2E7C04649
:10752000FF070000F0B55F464D4644465646F0B4AE
:107530001C03240BA4462F4C0F034D005E00C90F03
:1075400080463F0B6D0D8B469146760DDB0FA542B5
:1075500020D0284CA64222D0002D12D138434442DC
:107560004441002E20D0002C0DD05C426341012408
:107570005B421C4320003CBC90469946A246AB4669
:10758000F0BD002E17D05B4519D05B465C4201234D
:107590001C43EFE7390002240143EBD1D9E76146F0
:1075A00002241143E6D1D7E761460A43DBD1002428
:1075B0000028DFD0E9E761460A43E4D1E5E7B542B8
:1075C00003DD01225C421443D4E7B542CDDB6745BD
:1075D000DBD809D000246745CCD259464C426141E2
:1075E000012449420C43C5E7C845CED80024C8450C
:1075F000F3D3BFE7FF070000F0B55F4656464D46A0
:107600004446F0B40D0399464E002B0B87B007009B
:10761000924680469B46760DCC0F002E69D06D4B6E
:107620009E4235D05B468022DD001204430F134397
:107630002B439B46C3009846674B00279C4600237C
:10764000664401934A4615035000D20F53462D0B52
:10765000400D914600D176E05E4A90426CD0802287
:107660005B0F120413435C4AED0094461D435346DE
:107670000022DB00604449463618701C61400290CD
:1076800017430F2F00D9AFE05448BF00C759BF467A
:107690005B461F4300D088E000239B469846023398
:1076A00008270193CEE74946022A6AD0032A00D16F
:1076B00009E2012A00D0BBE111400022002300258D
:1076C0009046CCB200212D030A0D12052D0B154357
:1076D000434A1B0515401D436D00E4076D08254313
:1076E0004046290007B03CBC90469946A246AB46AE
:1076F000F0BD034352D05B46002B00D18AE15846CF
:1077000000F014FE03000B3B1C2B00DD7BE11D226F
:10771000D31A3A0001005D46DA4008398D40130063
:107720008F402B439B46B8462E4B00279C46002398
:1077300060444642019385E752462A432CD10025F6
:107740000023022297E752462A4321D0002D00D180
:1077500054E1280000F0EAFD03000B3B1C2B00DD88
:1077600046E11D21CB1A51460200D9405346083A42
:10777000954093400D431B4A94466044404200228A
:1077800079E7012400220C40124B0025904699E72E
:107790000025002301226EE703226CE700239B46AD
:1077A00098460133042701934CE703230C270193E8
:1077B00048E700238025984600242D03054B81E7E8
:1077C0005D464346019A6FE75D4643462100019AB4
:1077D0006AE7C046FF07000001FCFFFF30A8000079
:1077E000FFFF0F80F30300004246120C91461A0C73
:1077F0009446424617044A461B041B0C5A436046F3
:1078000090464A4642431000039262461C003F0CD9
:107810007A437C4342440192220C9246019A52449C
:10782000904506D98246802040028046C244504698
:107830000390100C049048462404240C12041219DE
:1078400005922A0C2D042D0C68432C0082464846D4
:107850007C4350438146200C80465743574447445D
:10786000BA4503D9802040028046C144380C3F0409
:10787000B84648442404240C01900498A044404491
:1078800004905846000C814658460404200C824659
:10789000070048465F434C464343604660436446A6
:1078A000834650464443380C8446E4186444A3425B
:1078B00003D980235B029C46E34448463F04230CE3
:1078C0003F0C2404E419574668436F4384464D46F1
:1078D000504655434243380C814662444A445B4417
:1078E000944503D9802040028446654403983F04B0
:1078F000834604983F0C8446E344C345804140429C
:107900008246100484460198674484466744A34431
:10791000BC46A345A4419946D44464428742BF4132
:10792000D4458041E144A04699459B417F42404275
:10793000C8440743120CBA18A045A4415F423B005B
:1079400064422343D71843467D19DB0D6D021D4366
:107950005B465A02059B1A43531E9A415B46DB0D58
:107960001A4343465B021343EA0107D501225C0830
:1079700013402343EA07029E13436D08574AB21887
:10798000002A4BDD580709D00F201840042805D0E5
:10799000181D98429B415B42ED180300E80104D595
:1079A0004F4A15408022D200B2184E48824200DD74
:1079B000E7E60124DB08680718436D02530580469B
:1079C0002D0B5B0D0C407DE68022594612031142BF
:1079D00008D0154206D115432D0398462D0B4C4671
:1079E000414B6FE65D4615432D032D0B3E4B69E67B
:1079F00003005546283B9D400023BCE6504600F05E
:107A000095FC2030A8E60300283B9F400023BB469E
:107A1000984689E600F08AFC203073E60124A61A15
:107A2000382E07DD00220C4000230025904649E651
:107A3000029EA3E71F2E20DC20222C001800921BA0
:107A4000F040944093400443581E83411C43F5404A
:107A5000630709D00F232340042B05D023001C1DEE
:107A60009C4292415242AD182B021FD501240022A4
:107A70000C4001230025904624E61F202C004042A4
:107A8000821AD440202E1CD04022961BB5402B4396
:107A9000581E83410720234318400025002809D0A1
:107AA0000F2200251A401C00042AD8D123006807A1
:107AB0006D022D0B0124DB08034398460C40002384
:107AC00000E60025E3E780220124120315432D037D
:107AD00098462D0B0C40044BF4E5C046FF03000014
:107AE000FFFFFFFEFE070000FF070000F0B557464E
:107AF0004E464546E0B40E001100F20F9246C50016
:107B0000420F180337037400400A4E0F7F0A3043B8
:107B1000CF4E17435A00640D520DDB0FC900B2421D
:107B200000D1E5E001267340A61AB446534500D1C2
:107B3000AFE0002E00DC0DE1002A3AD103000B4338
:107B400000D0E4E06B0709D00F232B40042B05D0B5
:107B50002B1DAB42AD416D427F191D003B0200D48D
:107B600088E0BB4B01349C4200D110E13A00B94B94
:107B700051461A4001235007ED085202640505439F
:107B8000120B640D0B400021280012030D0D120B87
:107B900064052D0515436208AF4CDB072C401443E8
:107BA000640064081C4321001CBC90469946A24610
:107BB000F0BDA74B9C42C5D080231B0418436346ED
:107BC000382B00DDFDE01F2B00DD30E16246202375
:107BD0009B1A02009A40664690460A009940F2407D
:107BE00046464B1E99413243114363460200DA4038
:107BF000691A8D429B410D00BA1A5B42D71A3B02AB
:107C000035D57A02530A98464346002B00D1C4E08A
:107C1000404600F08BFB0300083B1F2B00DDC5E056
:107C200020222900D21A4746D1409F400A009D4099
:107C30003A439C4200DDC0E01C1B631C1F2B00DD8F
:107C4000E4E0202114002800C91AD8408C408D405F
:107C50000443DA40681E854117002543002471E77C
:107C6000424663461A4300D14CE2674645466B07DD
:107C700000D069E7012351467807ED08FA080B4068
:107C8000054373498C4238D012036405120B640D0E
:107C900079E7002E00DC9AE0002A47D06C4A944233
:107CA00000D14FE78022120410436246382A00DCDC
:107CB00008E10143481E81410022C9B24919D21985
:107CC000A942BF410D007F42BF183A0200D442E1F1
:107CD0005F4A0134944200D14EE101205D4A6908B7
:107CE0003A4028400843D507054357089A4629E7F4
:107CF00006000E4300D017E714E72900114300D116
:107D0000F9E1802109030A431203120B3BE7012327
:107D10005B429846C4446346002B72D1691A8D4277
:107D20009B413F1A5B42FF1A0D0068E702000A43BD
:107D300000D107E7012252429046C4446246002A1D
:107D400000D0E6E06918A942B6413F187642F7191B
:107D50000D00BAE7002E00D080E0621C5205520DE3
:107D6000012A00DCF9E06A1A91464D45B6413A1AFB
:107D70007642921B9046120200D499E04D1BA94214
:107D80008941C71B49427A1A90469A463CE75246B7
:107D90000123002513400022F5E6280000F0C6FA72
:107DA00020300300083B1F2B00DC39E72A0028386D
:107DB000824000259C4200DC3EE7264FE41A174033
:107DC000C0E60143481E81410022C9B210E7002EDF
:107DD00000D0F1E0621C94465205520D012A00DCED
:107DE000A0E01B4A944500D1C5E06918A942924120
:107DF0003F185242D2194908D5070D435708644627
:107E0000A0E6134B9C4200D0D9E69BE611001F3C34
:107E1000E1400C00202B00D180E04021CB1A9A4099
:107E200015436A1E95410027254300241FE763463A
:107E30000200203BDA406346202B71D04023664687
:107E40009B1B98400143481E814111430022CFE60D
:107E5000FF070000FFFF7FFFFFFF0F80002C48D0CF
:107E6000CA4CA24200D1A2E07442A146802424045C
:107E700027434C46382C00DDDBE01F2C00DD44E1BD
:107E80004E462024A41B3E00A640A246B0464C46C7
:107E90002E00E640B4464646644626435446A54076
:107EA0006C1EA54134002C434D46EF400D1B28E0CD
:107EB0004A4643464D461A4300D0A5E60023002417
:107EC0000025DEE61F2A5ADC66462022921B0600A9
:107ED00096409146B04662460E00D6404246164352
:107EE0004A4691404A1E9141020060463143C240D9
:107EF000E4E63C002C435AD0F443A146002C52D176
:107F00004D1BA9428941C71B49427F1A14009A465A
:107F100075E69E4A944200D0C7E613E600227FE74A
:107F200000208FE7002C00D0C8E03B002B4300D19D
:107F30000FE103000B4300D104E66918A9429B41FD
:107F40003F185B42DF193B0200D41AE1904B0D0051
:107F50001F406446F6E59A4689E63A002A43002C1B
:107F60005CD1002A75D102000A4300D1CAE00700A3
:107F70000D009A46E6E564460022002581E6624649
:107F80000600203AD6406246B046202A00D1B7E02B
:107F900040226646921B904001434246481E814162
:107FA000114300228AE6794CA24200D061E7070023
:107FB0000D0014009A46C5E5002C41D13C002C432D
:107FC00078D0F443A146002C20D0704CA24271D04E
:107FD0004C46382C00DDB2E01F2C00DDBCE0202632
:107FE000341BA2463C005646B4404E46A0462C00E8
:107FF000F440A446444666463443A4465446A5404D
:1080000064466E1EB54125434C46E7406D188D42CF
:1080100089413F184942CF19140056E6002A2FD152
:1080200002000A4300D184E007000D009A46574C35
:1080300088E53D436F1EBD41ECB200270D1B60E794
:10804000524CA24236D0744280263604A1463743B1
:10805000BEE702000A4300D174E56A1A904645451E
:10806000B6413A1A7642921B9446120200D4F7E5C2
:108070004D1BA9428941C71B49427F1A9A4661E5B7
:1080800002000A433AD0ED087C072C438025FA0809
:108090002D032A4208D0C7082F4205D145072C00DE
:1080A0003A009A46C9080C43670FD200E50017430F
:1080B000364C47E507000D00140043E53A002A431B
:1080C00043D002000A4319D0ED087C072C438025D9
:1080D000FA082D032A4207D0C6082E4204D14707CA
:1080E0003C003200C9080C43D700620FE50017437B
:1080F0009A46264C26E50022002544E5234C21E53E
:10810000002049E700230025BBE54C463E00203C0B
:10811000E6404C46B446202C31D040244E46A61BA7
:10812000B7403D436C1EA54164462C4300270D1B00
:10813000E7E6802200231203144C0025A1E53D430D
:108140006F1EBD410027EDB260E707000D000F4C28
:10815000F8E407000D00F5E44E463C00203EF440F4
:10816000A0464C46202C0ED040244E46A41BA740CF
:108170003D436F1EBD4144460027254346E7002787
:10818000CFE70D0073E50027F2E7C046FF070000C8
:10819000FFFF7FFF0B0330B5134D1A0B4B005B0D38
:1081A000C90F0024AB4211DD104CA34210DC802427
:1081B000640322430E4CE41A1F2C0CDD0D48C31A35
:1081C000DA4013005C42002900D11C00200030BDC1
:1081D000094BCC18FAE7E040084CA44663449A40A7
:1081E00013000343EEE7C046FE0300001D04000039
:1081F0003304000013040000FFFFFF7FEDFBFFFFCF
:1082000070B5002830D0C317C4185C40C50F2000DB
:1082100000F08CF8174B184A1B1AD21A1F2A18DDC7
:10822000164AD21A9440002224035B05240B5B0DEE
:108230000021100024030A0D1205240B1443104AD8
:108240001B0514401C436400ED0764082C43210007
:1082500070BD210091400A000B21081AC4405B0543
:108260002403240B5B0DE3E70025002300240022F8
:10827000DEE7C0461E0400003304000013040000C3
:10828000FFFF0F804200120E511C4302C9B270B5AD
:108290005D0AC40F012915DDE02189008C466D07B8
:1082A0001B0B6244002128000D0D2D052B431C4D96
:1082B00052052B40520813435B00E4075B0823433D
:1082C000190070BD002A15D1002D1FD0280000F024
:1082D0002DF80A281DDC0B232A001B1ADA40130094
:1082E0000200153295400F4A1B03121A52051B0B50
:1082F000520DD7E7002D06D080221B0B120313432B
:108300006D07094ACEE7084A0023CBE70022002385
:10831000C8E703000B3B9D402B000025E3E7C04668
:10832000FFFF0F8089030000FF0700001C210123CD
:108330001B04984201D3000C10391B0A984201D348
:10834000000A08391B09984201D30009043902A226
:10835000105C40187047C04604030202010101018D
:1083600000000000000000007FB51D000A4B060061
:108370001B68D868002A02D1084C230001E01300D2
:10838000074C0293009133002A000649019400F043
:1083900021F800F023FEC0468002002032A2000037
:1083A00070A800007DA80000084B10B50400002B49
:1083B00002D0002100E000BF054B1868836A002B43
:1083C00000D09847200001F0F3FAC04600000000FA
:1083D000B0A800000EB403B5010003AB044804CB01
:1083E0000068019300F016F902B008BC03B018470A
:1083F000800200200E4B70B500251E000D4CE41AC3
:10840000A410A54204D0AB00F35898470135F8E713
:1084100001F0D0FA084B00251E00084CE41AA41005
:10842000A54204D0AB00F35898470135F8E770BD7A
:108430008802002088020020880200209802002084
:1084400010B5034B0100186800F066F810BDC04677
:108450008002002010B5034B0100186800F016F8E8
:1084600010BDC04680020020002310B59A4203D000
:10847000CC5CC4540133F9E710BD03008218934269
:1084800002D019700133FAE77047000030B50029B7
:108490003ED004390B68002B00DAC9181D4A136856
:1084A0001400002B02D14B60116031E08B420DD9DA
:1084B0000A688818834203D118685B6882180A60CA
:1084C0004B60216024E08A4203D813005A68002AD6
:1084D000F9D11D685C198C420BD1096869185818CC
:1084E0001960824214D110685268411819605A60AC
:1084F0000EE08C4202D90C23036009E008680C18D6
:10850000A24203D114685268201808604A6059607A
:1085100030BDC046D8110020032370B5CD1C9D434B
:10852000083506000C2D01D20C2505E0002D03DADC
:108530000C230020336040E0A942F9D81F4B1C688F
:108540001A002100002913D00B685B1B0DD40B2BE4
:1085500002D90B60CC181EE08C4202D16368136014
:108560001AE04B6863600C0016E00C004968E9E70C
:10857000134C2368002B03D1300000F033FB206044
:108580002900300000F02EFB431CD1D00323C41C73
:108590009C43A0420AD12560200007220B30231DF6
:1085A0009043C31A09D05A42E25006E0211A300023
:1085B00000F018FB431CEED1BAE770BDD8110020C3
:1085C000D4110020936810B5013B9360002B05DAAD
:1085D0009469A34208DBCBB20A2B05D01368581C60
:1085E00010601970C8B201E000F02CFC10BDF8B5A5
:1085F00006000F001400D518AC4208D021783A00CC
:108600003000FFF7DFFF0134431CF5D100E000200C
:10861000F8BD0000F0B59FB006000F000292059370
:10862000002804D08369002B01D100F0D3FD7F4BDB
:108630009F4201D1776808E07D4B9F4201D1B76826
:1086400003E07C4B9F4200D1F768BB891B070AD52A
:108650003B69002B07D0002306AD6B6120336B769E
:108660001033AB763DE03900300000F043FC0028C9
:10867000F1D001204042D6E0059A111D1268059103
:10868000002A00DA7FE00992013423782E2B00D1F2
:108690008DE021780322684800F082FE002807D090
:1086A000654B2A68C01A4023834013432B60013472
:1086B0002178631C062261480293297600F070FE3F
:1086C000002800D19DE05E4B002B00D090E00722F7
:1086D000059B07339343083305936B69039A9B18F3
:1086E0006B61029C2378002B04D1029BE31A049354
:1086F00012D003E0252BF8D00134F3E7049B029A53
:1087000039003000FFF773FF431C00D186E06A692F
:10871000049B944663446B612378002B7ED0012236
:10872000002352426A6002A95432521801342B606D
:10873000EB60AB601370AB6521780522414800F017
:108740002FFE002808D03F4B2A68C01A012383401F
:1087500013432B600134EFE72B68DA0604D553226C
:10876000202102A8121811701A0704D553222B21B8
:1087700002A81218117022782A2A00D17CE7099BDE
:1087800000200A2105E05242EA60022213432B60D6
:108790007AE72278303A092A04D84B4301349B18EF
:1087A0000120F6E7002800D16FE709936DE76378B1
:1087B0002A2B0AD1059B02341A1D1B680592002B37
:1087C00001DA01235B42079363E700230A201A00C2
:1087D00001346B6021783039092904D842430134CF
:1087E00052180123F6E7002B00D152E7079250E719
:1087F00005AB00933A00144B2900300000E000BFA5
:1088000007E005AB00933A000F4B2900300000F061
:108810008BF80390039B013300D05EE7BB895B06B6
:1088200000D526E70B981FB0F0BDC046E8A90000B0
:1088300008AA000028AA0000BAA80000BEA80000EC
:1088400000000000B4A80000EF850000F7B5170095
:1088500001938A680B6900900C00934200DA1300C0
:1088600022003B6043321278002A01D001333B6082
:1088700023689B0602D53B6802333B6006252368CC
:108880001D401ED0230043331B785A1E934122689B
:1088900092061CD53020E1184331087021005A1C83
:1088A00045310978A2184332023311700FE02200DB
:1088B0000123193201990098089EB047431C0ED03D
:1088C0000135E3683A689B1A9D42F0DBDAE7220043
:1088D000019943320098089DA847431C02D101200A
:1088E000404220E006232068E1683A680340002502
:1088F000042B03D18D1AEB43DB171D40A3682269BB
:10890000934201DD9B1AED180027BD420AD02200D8
:1089100001231A3201990098089EB047431CDED00B
:108920000137F2E70020FEBDF0B58BB006920A00D9
:1089300043320793059004920A7E0C00109B6E2A26
:1089400000D1ABE011D8632A22D009D8002A00D187
:10895000B5E0582A00D0C5E045310A70814A4FE0A1
:10896000642A1DD0692A1BD0BCE0732A00D1AAE07A
:1089700009D86F2A29D0702A00D0B3E020220968D4
:108980000A43226037E0752A1FD0782A33D0A9E045
:108990000E001A684236111D196013683370A4E086
:1089A00021681A68080606D4490604D5111D196005
:1089B0000023D55E02E0111D19601568002D3BDA19
:1089C0002D23049A6D42137036E021681A68080658
:1089D00006D4490604D51568111D1960ADB202E030
:1089E000111D196015685F4B227E039308276F2ABB
:1089F0001DD00A271BE022007821453211705A4A07
:108A000019680392081D226818600D68100602D4C8
:108A1000500600D5ADB2D30702D520231A432260F9
:108A20001027002D03D1202322689A4322602300BF
:108A3000002243331A7002E00A274A4B039363680B
:108A4000A360002B09DB0422216891432160002DE3
:108A500005D1049E002B11D07BE0002D79D0049E1F
:108A600028003900FDF7CAFE039B013E5B5C28002D
:108A700033703900FDF73CFE051EF1D1082F09D1F6
:108A80002368DB0706D563682269934202DC302342
:108A9000013E3370049B9B1B23612BE009681A681D
:108AA000080607D4490605D5111D19601368A28A66
:108AB0001A8004E0111D1960136862691A600023AE
:108AC000049E236116E01A68111D196016680021C2
:108AD0006268300000F064FC002801D0801B6060F8
:108AE000636803E0260042363270012323610023CD
:108AF000049A1370079B09AA00932100069B05980E
:108B0000FFF7A4FE431C02D10120404227E0236965
:108B1000320006990598079DA847431CF4D02368A6
:108B200000259B070FD4099BE068984217DA1800CC
:108B300015E022000123193206990598079EB047D7
:108B4000431CE1D00135E368099A9B1A9D42F0DB92
:108B5000E9E72600039B42361B7833708EE70BB0A3
:108B6000F0BDC046C5A80000D6A80000154B10B542
:108B70001C68A36B002B15D11820FFF761FC124B6A
:108B8000A0630380114B01224380114B8380114B62
:108B9000C380114B03810523438106338381002366
:108BA00002614361A46B0D4A206961690C4BFDF7BA
:108BB00061FF012200238018594120616161480052
:108BC000400810BD800200200E330000CDABFFFF37
:108BD000341200006DE6FFFFECDEFFFF2D7F954CA9
:108BE0002DF45158002370B5064C05000800236091
:108BF00000F0C8FE431C03D12368002B00D02B607B
:108C000070BDC046F02500200CB430B5164B9DB0A9
:108C10000C1E1D6804DA8B2301202B6040421DE0EE
:108C2000822302A99B008B810023029008619C4251
:108C300000D0631E8B604B6101235B42CB81209A85
:108C400021AB2800019300F053FC431C01DA8B2375
:108C50002B60002C02D00023029A13701DB030BC90
:108C600008BC02B01847C046800200200EB410B500
:108C70009DB002A9029008610B4882248860486177
:108C8000012040421FABC881084804CBA400006803
:108C900001938C8100F02CFC0023029A13701DB00C
:108CA00010BC08BC03B01847FFFFFF7F8002002004
:108CB00002780B78002A03D0013001319A42F7D0B4
:108CC000D01A7047031C0A7801311A700133002A48
:108CD000F9D170470023C25C0133002AFBD1581E32
:108CE0007047030030B5002A0DD00C7801335D1EAB
:108CF000013A2C700131002CF5D19A189A4202D019
:108D00001C700133FAE730BDF0B51E00454B87B04B
:108D10001B680192029308220B00059003911C78B6
:108D200002995D1C09194878104001D02B00F6E724
:108D30002D2C04D19D1C5C780123009304E000904D
:108D40002B2C01D15C789D1C002E02D0102E0AD154
:108D500062E0302C5ED120222B789343582B54D1E3
:108D600010266C780235009F31007B1E9F412E4BF0
:108D7000FF183800FDF742FD380004913100FDF77F
:108D8000B7FC00230322070094461800029A121928
:108D900051780422114201D0303C07E06246114074
:108DA00017D03722012900D02032A41AA64210DDA4
:108DB0005A1C0BD0B84207D802D1049B9C4203DC5A
:108DC00070430123201801E001235B422C78013518
:108DD000DCE75A1C0BD10098059A431E9841124BB0
:108DE000C01822231360019B002B0AD117E0009AC0
:108DF000002A00D04042019A002A10D0039A002B8A
:108E000000D06A1E019B1A6009E03024002EAAD10E
:108E10000826A8E70A26A6E7302C9CD0A3E707B0CF
:108E2000F0BDC04684020020FFFFFF7F10B5130095
:108E30000A00010002480068FFF766FF10BDC04647
:108E400080020020F8B505000F001400002804D0AF
:108E50008369002B01D100F0BDF9234B9C4201D165
:108E60006C6808E0214B9C4201D1AC6803E0204BC8
:108E70009C4200D1EC68A369A360A3891B070AD5B3
:108E80002369002B07D023682269FEB2981A636910
:108E900098420FDB08E02100280000F02BF80028A2
:108EA000F1D0012040421DE02100280000F024F90B
:108EB0000028F6D1A3680130013BA36023685A1C47
:108EC00022601F706369984205D0A3893000DB07D8
:108ED00008D50A2E06D12100280000F00DF900283F
:108EE000DFD13000F8BDC046E8A9000008AA0000A4
:108EF00028AA0000354B70B51D6806000C00002D37
:108F000005D0AB69002B02D1280000F063F9304B8B
:108F10009C4201D16C6808E02E4B9C4201D1AC68A8
:108F200003E02D4B9C4200D1EC68A3899AB2110753
:108F300023D4D10607D409220120326037321343EB
:108F4000A381404240E0530713D5616B002908D04C
:108F500023004433994202D03000FFF797FA0023F0
:108F600063632422A3899343A3810023636023695D
:108F700023600822A3891343A3812369002B0BD10B
:108F8000A023A2899B00134080229200934203D029
:108F90002100300000F0B2F90123A289134005D06E
:108FA0000023A36063695B42A36103E0910700D4DF
:108FB0006369A36000202369834205D1130603D5AA
:108FC00040231A43A281013870BDC04680020020B0
:108FD000E8A9000008AA000028AA000010B5062091
:108FE00000F0AEFB012000F0E3FC0000F7B58A8939
:108FF00005000C0013075AD44B68002B02DC0B6CE5
:10900000002B19DDE76A002F16D000232E682B6095
:1090100080235B011A4001D0606D14E00123216AB6
:109020002800B847431C0ED12B68002B0BD01D2BFA
:1090300001D0162B02D12E6000205AE04022A389D5
:109040001343A38155E0A3895B0706D56368C01A63
:10905000636B002B01D0236CC01A00230200216A2D
:109060002800E76AB847A389421C06D129681D2950
:109070003AD8204ACA40D20736D500226260226917
:109080002260DB0405D5431C02D12B68002B00D1E4
:109090006065616B2E600029CED023004433994275
:1090A00002D02800FFF7F2F90020606321E00F6989
:1090B000002FC1D00B680F60DB1B019300239207C8
:1090C00000D14B69A36003E0019B3F181B1A019379
:1090D000019B002BB0DD019B3A00216A2800A66AA3
:1090E000B0470028F0DCA389402201201343A3816C
:1090F0004042FEBD010040200B6970B505000C0028
:10910000002B01D100201CE0002804D08369002B33
:1091100001D100F05FF80B4B9C4201D16C6808E074
:10912000094B9C4201D1AC6803E0084B9C4200D142
:10913000EC680C22A35E002BE4D021002800FFF78E
:1091400055FF70BDE8A9000008AA000028AA000089
:1091500010B5024900F0B0F810BDC046F99000000B
:10916000002310B50400036043608360818143667F
:10917000C281036143618361190008225C30FFF7FB
:109180007CF9054B24626362044BA362044BE362E7
:10919000044B236310BDC04681970000A9970000CF
:1091A000E19700000D98000070B568254B1E5D43E7
:1091B0000E0029007431FFF7AFF9041E08D000211A
:1091C0002A00016046600C30A0606832FFF755F954
:1091D000200070BD836913B50400002B28D183647F
:1091E000C3640365134B144A1B688262019398425F
:1091F00001D101238361200000F020F8606020008D
:1092000000F01CF8A060200000F018F80022E060D8
:1092100004216068FFF7A4FF01220921A068FFF77D
:109220009FFF02221221E068FFF79AFF0123A3614A
:1092300013BDC046B0A8000051910000F8B51D4B09
:1092400006001D68AB69002B02D12800FFF7C2FFA2
:109250004835AC686B68013B05D40C22A75E002F33
:1092600010D06834F7E72B68002B01D02D68F0E7A9
:1092700004213000FFF798FF28600028F6D10C2366
:10928000336016E0012320005B42E3810233A381B7
:1092900067662760A760676027616761A7615C30C8
:1092A00008223900FFF7E9F820006763A763A76485
:1092B000E764F8BDB0A80000F7B504000700002679
:1092C00001914834002C16D06368A5680093009B78
:1092D000013B00930DD4AB89012B08D90E22AB5E64
:1092E000013304D029003800019B984706436835B4
:1092F000EDE72468E6E73000FEBD0000F0B58B899D
:1093000091B006000C009B0726D40E23C95E0029ED
:1093100004DA8023A5891D4010D10CE001AA00F0D9
:10932000A1FA0028F5DBF023029D1B021D401A4B19
:10933000ED186B425D418027FF0001E000254027CA
:1093400039003000FFF7E8F800280CD1A3899A050E
:109350001FD402221343A3812300473323602361D8
:109360000123636115E080220C4BB362A389206066
:109370001343A38120616761002D0AD00E23E15EB3
:10938000300000F081FA002803D00122A3891343A2
:10939000A38111B0F0BDC04600E0FFFF5191000075
:1093A000C9B28218904204D003788B4202D00130B7
:1093B000F8E70020704710B5884202D98B18984210
:1093C00001D3002305E09B1A013A08D3995C81542C
:1093D000FAE7934203D0CC5CC4540133F9E710BDE3
:1093E000F8B506000C001500002904D11100FFF7A4
:1093F00093F8040018E0002A03D1FFF747F82C0087
:1094000012E000F067FA85420ED929003000FFF71C
:1094100083F8071E07D021002A00FFF725F8210056
:109420003000FFF733F83C002000F8BDF0B58E683F
:1094300085B007000C00039201939E4243D890230D
:109440008A89DB001A423ED0032509692368019806
:109450005B1A029363695D43EB0F5D19029B6D100C
:1094600001331B18AB4200D91D00530510D529004C
:109470003800FFF751F8061E14D0029A2169FEF752
:10948000F3FFA289194B134080221343A38112E0FA
:109490002A003800FFF7A4FF061E0CD1216938000E
:1094A000FEF7F4FF0C23402201203B60A3894042D9
:1094B0001343A38117E0029B2661F61826606561BD
:1094C000019EED1AA560019BB34200D21E0032003E
:1094D00003992068FFF76FFF0020A3689B1BA36020
:1094E00023689E19266005B0F0BDC0467FFBFFFFD4
:1094F000F0B59FB0029005938B890F0016001B06F4
:1095000010D50B69002B0DD14021FFF705F838600D
:109510003861002804D10C23029A01381360D8E086
:1095200040237B61002306AD6B6120336B761033E3
:10953000AB7634002378002B03D1A31B049312D005
:1095400003E0252BF9D00134F4E7A31B32003900E6
:109550000298FFF76BFF431C00D1B4E06A69049BDB
:10956000944663446B612378002B00D1ABE0012269
:10957000002352426A6002A95432521801342B600F
:10958000EB60AB601370AB65534E21780522300061
:10959000FFF706FF002807D00123801B83402A68BD
:1095A000013413432B60EFE72B68DA0604D553220E
:1095B000202102A8121811701A0704D553222B215A
:1095C00002A81218117022782A2A03D0099B0020C1
:1095D0000A210EE0059A111D12680591002A01DB8F
:1095E000099204E05242EA60022213432B600134E4
:1095F0000BE02278303A092A04D84B4301349B18F7
:109600000120F6E7002800D0099323782E2B1ED1E5
:1096100063782A2B0AD1059B02341A1D1B68059218
:10962000002B01DA01235B42079310E000230A209C
:109630001A0001346B6021783039092904D842437B
:10964000013452180123F6E7002B00D00792234E75
:10965000217803223000FFF7A3FE002806D0402324
:10966000801B83402A68013413432B602178062233
:109670001B48661C2976FFF793FE002812D0194B71
:10968000002B06D10722059B07339343083305932C
:1096900014E005AB00933A00134B2900029800E058
:1096A00000BF07E005AB00933A000F4B290002987A
:1096B000FFF73AF90390039B013304D06B69039AD7
:1096C0009B186B6135E7BB890B985B0601D50120C0
:1096D00040421FB0F0BDC046B4A80000BAA80000C8
:1096E000BEA80000000000002D94000070B504002A
:1096F0000D1E1F2D04D916230360012040421EE0D9
:10970000426C002A04D08B00D2181368002B08D1B9
:10971000200000F031F82A000100200000F01AF8C3
:109720000DE00020012B0AD0591C03D11733236010
:10973000013004E00024280014609847200070BD28
:1097400010B5034B01001868FFF7D0FF10BDC046ED
:1097500080020020002370B5064C050008001100AF
:10976000236000F0F7F8431C03D12368002B00D0DE
:109770002B6070BDF025002010B500F0DBF810BDA7
:1097800070B50C000E25495F00F0B0F8002803DB2F
:10979000636D1B18636503E0A289024B1340A3812C
:1097A00070BDC046FFEFFFFFF8B51F008B890500B5
:1097B0000C001600DB0505D50E23C95E002202232E
:1097C00000F074F8A289054B28001340A3813200F1
:1097D0000E23E15E3B0000F01FF8F8BDFFEFFFFF36
:1097E00070B50C000E25495F00F060F8A389421C9B
:1097F00003D1054A1340A38104E0802252011343A0
:10980000A381606570BDC046FFEFFFFF10B50E235A
:10981000C95E00F015F810BD70B505000800110014
:109820000022064C22601A0000F0BAF8431C03D153
:109830002368002B00D02B6070BDC046F0250020AF
:10984000002370B5064C05000800236000F062F8A4
:10985000431C03D12368002B00D02B6070BDC04691
:10986000F0250020002370B5064C0500080011000B
:10987000236000F057F8431C03D12368002B00D06D
:109880002B6070BDF0250020002370B5064C05004C
:109890000800236000F056F8431C03D12368002B16
:1098A00000D02B6070BDC046F025002070B50500CB
:1098B000080011000022064C22601A0000F052F845
:1098C000431C03D12368002B00D02B6070BDC04621
:1098D000F02500200B1F1A68101F002A04DA8918CF
:1098E00004390B68D01804387047000070B50500C3
:1098F000080011000022064C22601A0000F03AF81D
:10990000431C03D12368002B00D02B6070BDC046E0
:10991000F025002058220120014B40421A60704778
:10992000F025002058220120014B40421A60704768
:10993000F025002058220120014B40421A60704758
:10994000F02500205822024B00201A607047C046C4
:10995000F025002058220120014B40421A60704738
:10996000F025002058220120014B40421A60704728
:10997000F025002058220120014B40421A60704718
:10998000F0250020044A1368002B03D0181810603B
:1099900018007047014BF9E7DC110020F825002082
:1099A00058220120014B40421A607047F0250020E8
:1099B000FEE7C046F8B5C046F8BC08BC9E467047F6
:1099C000F8B5C046F8BC08BC9E46704766616C732B
:1099D000650074727565006C697374206F6620256C
:1099E00064206974656D73006F626A656374206FCB
:1099F0006620636C6173733A20256400537461635D
:109A00006B20756E646572666C6F770036060000B9
:109A1000C8050000460600007C060000B8060000ED
:109A2000F20600002E070000560700009407000011
:109A3000DA070000360800007C080000FA08000081
:109A4000360900005E09000098090000E2090000E4
:109A50000A0A0000420A00007C0A0000B80A00005E
:109A60003E0B0000060C0000900C0000EE0C000005
:109A7000380D00005A0D00007E0D0000620E00003F
:109A8000AE0E000036060000360600003606000066
:109A90002A0F0000B20F00001C100000661000002A
:109AA000B41000003A110000C211000010120000B2
:109AB0005A12000090120000E4120000301300005F
:109AC0007C130000D813000034140000721400004E
:109AD000DE1400001615000062150000AE1500002F
:109AE000FA1500003416000080160000D41600009D
:109AF0003606000036060000360600003C1700005F
:109B000074170000AC170000DA17000012180000EC
:109B10004018000036060000360600003606000039
:109B20003606000078180000C01800003606000055
:109B3000360600000C1900003A19000084190000D4
:109B4000360600003606000036060000B219000096
:109B5000E2190000121A0000421A0000881A0000E0
:109B6000C01A0000EC1A0000161B0000401B000089
:109B7000701B0000A01B0000CC1B0000F81B0000A5
:109B8000281C0000541C00003606000036060000A9
:109B9000360600003606000036060000841C000071
:109BA000B21C0000E01C00000E1D00003C1D000067
:109BB000741D0000AC1D0000E41D00001C1E000010
:109BC000541E0000821E0000BA1E0000360600006F
:109BD0003606000036060000360600003606000095
:109BE0003606000036060000360600003606000085
:109BF0003606000036060000360600003606000075
:109C000036060000E81E0000161F000007000000D6
:109C10000300000043616C6C696F706500686173DC
:109C2000546F6E6500706C6179546F6E6500686189
:109C300073536572766F00736574536572766F0047
:109C400015000000010000000200000004000000F8
:109C500005000000060000000D0A564D2050616E00
:109C600069633A2025730D0A00496E73756666694B
:109C70006369656E74206D656D6F727920666F72B1
:109C8000204D6963726F426C6F636B73206F626A01
:109C9000656374206865617000496E7375666669F6
:109CA0006369656E74206D656D6F727920666F7281
:109CB000204D6963726F426C6F636B7320737461C4
:109CC000636B00626164206F626A65637420617413
:109CD00020256C640A0025783A20256420776F726D
:109CE00064732C20636C61737349442025640A00FB
:109CF0004865616465723A2025780A000930782544
:109D0000782C0A006D69736300686578546F496E3A
:109D1000740073696E006E657400686173576946FC
:109D200069007374617274576946690073746F7067
:109D30005769466900776966695374617475730081
:109D40006D79495041646472657373007468696E1B
:109D5000674465736372697074696F6E00636C65E4
:109D600061725468696E674465736372697074697F
:109D70006F6E00617070656E64546F5468696E67D1
:109D80004465736372697074696F6E0061707065A9
:109D90006E64546F5468696E6750726F7065727448
:109DA00079000D0E0F04050C0B0A060708090D0EAD
:109DB0000F04050C0B0A06070809646973706C61CF
:109DC00079006C696768744C6576656C006D6244F7
:109DD0006973706C6179006D62446973706C61794C
:109DE0004F6666006D62506C6F74006D62556E70E8
:109DF0006C6F74006D6244726177536861706500C6
:109E00006D625368617065466F724C6574746572FB
:109E1000006E656F506978656C53656E64006E65A1
:109E20006F506978656C53657450696E000000006E
:109E3000000000000100000002000000030000001C
:109E400004000000050000000600000007000000FC
:109E500008000000090000000A0000000B000000DC
:109E60000C0000000D0000000E0000000F000000BC
:109E70001000000012000000140000001600000096
:109E8000180000001A0000001C0000001E00000066
:109E90002000000023000000260000002900000030
:109EA0002C0000002F0000003200000036000000EF
:109EB0003A0000003E0000004200000046000000A2
:109EC0004B00000050000000550000005A00000048
:109ED00061000000680000006F00000076000000D4
:109EE0007D000000840000008B0000009200000054
:109EF00099000000A0000000A7000000AE000000D4
:109F0000B5000000BC000000C3000000CA00000053
:109F1000D1000000D8000000DF000000E6000000D3
:109F2000ED000000F4000000FB000000FF00000056
:109F3000000000000008080800080A4A4000000A63
:109F40005FEA5FEA0ED92ED36E19324489330C9240
:109F50004C924D0808000000048808080408048496
:109F60008488000A448A4000048EC48000000004F3
:109F70008800000EC0000000000800012244881084
:109F80000C9252524C048C84848E1C824C901E1E67
:109F9000C244924C06CA525FE21FF01EC13E024408
:109FA0008ED12E1FE24488100ED12ED12E0ED12E2E
:109FB000C488000800080000048004880244880463
:109FC00082000EC00EC008048244880ED126C00450
:109FD0000ED135B36C0C925ED2521C925C925C0E28
:109FE000D010100E1C9252525C1ED01C901E1ED01F
:109FF0001C90100ED013712E12525ED2521C880883
:10A00000081C1FE242524C12549814921010101067
:10A010001E113B75B131113935B3710C9252524C4E
:10A020001C925C90100C92524C861C925C92510EC9
:10A03000D00C825C1FE4848484125252524C113141
:10A04000312A44113135BB7112524C9252112A44BB
:10A0500084841EC488101E0EC808080E10080482CE
:10A06000410EC242424E048A400000000000001F20
:10A070000804800000000ED2524F10101C925C00A9
:10A080000ED0100E02424ED24E0C925C900E06C8BC
:10A090001C88080ED24EC24C10101C9252080008A8
:10A0A0000808024002424C1014981492080808084C
:10A0B00006001B75B131001C925252000C92524C9A
:10A0C000001C925C90000ED24EC2000ED010100008
:10A0D00006C8049808080EC807001252524F001113
:10A0E000312A4400113135BB00124C8C9200112AE8
:10A0F0004498001EC4881E06C48C8486080808087C
:10A100000818080C881800000C836025642025645A
:10A110002025642025640A00436F6D7061637465B7
:10A120006420466C61736820636F64652073746F8C
:10A1300072650A256420627974657320757365649D
:10A1400020282564252529206F66202564002564A4
:10A150002025642025642028256420776F7264738D
:10A1600029002564207265636F7264732C20256456
:10A1700020776F7264732C206D61784944202564C8
:10A180002C20636F6D70616374696F6E20637963F7
:10A190006C657320256400426164207265636F7290
:10A1A0006420666F756E6420647572696E672069DD
:10A1B0006E697469616C697A6174696F6E210A00F5
:10A1C0004E6F7420656E6F75676820726F6F6D20BB
:10A1D0006576656E20616674657220636F6D70616F
:10A1E0006374696F6E0A00526573746F72656420E0
:10A1F00025642073637269707473005374617274A0
:10A200006564005363726970747320636C65617276
:10A210006564002D2D2D2D2D0A0050657273697314
:10A2200074656E74204D656D6F727920546573741A
:10A230000A0A000A496E697469616C697A696E6715
:10A24000204D656D6F72790A004D656D6F727920D2
:10A25000696E74697469616C697A65643B207772B0
:10A260006974696E67207265636F7264732E2E2E37
:10A270000A005265636F7264206174206F666673B2
:10A2800065742025643A20256420256420256420F7
:10A2900025642028256420776F726473290A00469C
:10A2A000696E616C3A2063757272656E7420256404
:10A2B0002075736564202564206330202564206345
:10A2C000312025640A006E6F6E6500726164696FEB
:10A2D0000064697361626C65526164696F006D65E9
:10A2E0007373616765526563656976656400706163
:10A2F000636B657452656365697665007061636B55
:10A30000657453656E64007265636569766564495A
:10A310006E74656765720072656365697665644D24
:10A32000657373616765547970650072656365690B
:10A33000766564537472696E670073656E64496E06
:10A3400074656765720073656E645061697200734D
:10A35000656E64537472696E6700736574436861F7
:10A360006E6E656C0073657447726F75700073650F
:10A3700074506F776572007369676E616C537472A5
:10A38000656E677468004E6F206672656520746143
:10A39000736B20656E7472696573004D656D6F72C5
:10A3A0007920636C656172656400416C6C20746136
:10A3B000736B732073746F7070656400763036341D
:10A3C000002025732025730073656E736F72730010
:10A3D00074656D70657261747572650074696C7412
:10A3E000580074696C74590074696C745A00746F05
:10A3F0007563685265616400693263526561640027
:10A4000069326357726974650074667400656E61C1
:10A41000626C65446973706C61790073657450692E
:10A4200078656C006C696E65007265637400726FAC
:10A43000756E6465645265637400636972636C650C
:10A4400000747269616E676C65007465787400747D
:10A450006674546F756368656400746674546F75D0
:10A4600063685800746674546F7563685900746645
:10A4700074546F75636850726573737572650057B5
:10A48000656C636F6D6520746F204D6963726F42F8
:10A490006C6F636B732100535049436C6173733A63
:10A4A0003A535049436C617373284E52465F535080
:10A4B000495F547970652A2C2075696E74385F7411
:10A4C0002C2075696E74385F742C2075696E743831
:10A4D0005F742900705F73706920213D204E554CD8
:10A4E0004C002F55736572732F6A6F686E6D616CC7
:10A4F0006F6E65792F4C6962726172792F41726457
:10A5000075696E6F31352F7061636B616765732F8D
:10A5100073616E646565706D69737472792F6861BB
:10A520007264776172652F6E5246352F302E362E4B
:10A53000302F6C69627261726965732F5350492FB5
:10A540005350492E637070000000000000000000AE
:10A55000DF470000A5470000CB470000D5470000BB
:10A5600005480000C947000000000000010000008D
:10A5700002000000160000000400000005000000BA
:10A5800006000000070000000800000009000000AD
:10A590000A0000000B0000000C0000000D0000008D
:10A5A0000E0000000F0000001A0000001B00000059
:10A5B0001400000013000000110000000300000060
:10A5C000100000001C0000001D0000001E00000024
:10A5D0001200000015000000170000001800000025
:10A5E00019000000FB21F93FFB2109407CD91240F2
:10A5F000FB2119407A6A1F407CD92240BBFD2540CF
:10A60000FB2129403A462C407A6A2F405C47314072
:10A610007CD932409C6B3440BBFD3540DB8F3740EA
:10A62000FB2139401BB43A403A463C405AD83D40A1
:10A630007A6A3F404C7E40405C4741406C1042404B
:10A640007CD942408CA243409C6B4440AC34454092
:10A65000BBFD4540CBC64640DB8F4740EB584840EA
:10A66000FB21494083F9A200444E6E00FC291500ED
:10A67000D1572700DD34F50062DBC0003C9995001E
:10A68000419043006351FE00BBDEAB00B761C500E3
:10A690003A6E2400D24D42004906E00009EA2E003D
:10A6A0001C92D100EB1DFE0029B11C00E83EA70062
:10A6B000F535820044BB2E009CE98400B42670006E
:10A6C000417E5F00D6913900538339009CF43900F4
:10A6D0008B5F840028F9BD00F81F3B00DEFF970068
:10A6E0000F980500112FEF000A5A8B006D1F6D00A7
:10A6F000CF7E360009CB2700464FB7009E663F004D
:10A700002DEA5F00BA277500E5EBC7003D7BF1003D
:10A71000F739070092528A00FB6BEA001FB15F0015
:10A72000085D8D00300356007BFC4600F0AB6B00EB
:10A7300020BCCF0036F49A00E3A91D005E619100B1
:10A74000081BE60085996500A0145F008D40680035
:10A7500080D8FF0027734D0006063100CA56150049
:10A76000C9A873007BE260006B8CC000020000008F
:10A7700003000000040000000600000000000000CC
:10A7800000000040FB21F93F000000002D44743E12
:10A79000000000809846F83C0000006051CC783BF7
:10A7A00000000080831BF0390000004020257A382B
:10A7B000000000802282E336000000001DF36935AE
:10A7C00000000000000000009D5F00008D5D0000A3
:10A7D0000D6000002160000017600000995F00001C
:10A7E0008D5F00002D600000B95F0000895F0000F0
:10A7F000E86B0000466B0000466B0000446B0000F5
:10A80000DA6B0000DA6B0000D06B0000446B0000D4
:10A81000DA6B0000D06B0000DA6B0000446B0000C4
:10A82000E06B0000E06B0000E06B00006A6C000071
:10A83000E8770000A8760000A8760000A676000061
:10A84000C0770000C0770000B2770000A676000055
:10A85000C0770000B2770000C0770000A676000045
:10A86000C8770000C8770000C8770000C8790000EA
:10A870002C2066756E6374696F6E3A200061737385
:10A88000657274696F6E2022257322206661696C7F
:10A8900065643A2066696C6520222573222C206C41
:10A8A000696E65202564257325730A004300000046
:10A8B00020020020232D302B2000686C4C006566A0
:10A8C0006745464700303132333435363738394101
:10A8D0004243444546003031323334353637383917
:10A8E0006162636465660000202020202020202013
:10A8F0002028282828282020202020202020202030
:10A90000202020202020202088101010101010104F
:10A910001010101010101010040404040404040497
:10A920000404101010101010104141414141410128
:10A930000101010101010101010101010101010107
:10A940000101011010101010104242424242420216
:10A9500002020202020202020202020202020202D7
:10A960000202021010101020000000000000000081
:10A9700000000000000000000000000000000000D7
:10A9800000000000000000000000000000000000C7
:10A9900000000000000000000000000000000000B7
:10A9A00000000000000000000000000000000000A7
:10A9B0000000000000000000000000000000000097
:10A9C0000000000000000000000000000000000087
:10A9D0000000000000000000000000000000000077
:10A9E0000000000000000000000000000000000067
:10A9F0000000000000000000000000000000000057
:10AA00000000000000000000000000000000000046
:10AA10000000000000000000000000000000000036
:10AA20000000000000000000000000000000000026
:10AA30000000000000000000000000000000000016
:0CAA40000000000000000000000000000A
:08AA4C002857FF7F0100000004
:10AA5400FFFFFFFF400600001D9C0000F51F0000E3
:10AA6400259C0000F11F00002E9C0000F91F00002F
:10AA7400379C0000FD1F0000099D000041240000D8
:10AA8400129D0000952400001A9D0000712500000D
:10AA9400229D0000892500002C9D000093250000C4
:10AAA400359D00009D250000409D0000A725000065
:10AAB4004C9D0000B12500005D9D0000BB250000F9
:10AAC400739D00007F2500008C9D0000752500000B
:10AAD400C29D0000E1250000CD9D0000A12A0000D8
:10AAE400D79D0000B5270000E49D0000D527000095
:10AAF400EB9D000025280000F49D0000752800004F
:10AB0400009E0000CD2A0000119E0000DD290000F7
:10AB14001E9E0000AD29000018000000D1A2000014
:10AB240001350000DEA2000005350000EEA20000A1
:10AB340009350000FCA200000D35000007A3000049
:10AB4400C934000017A30000DD3400002BA300006B
:10AB5400CD3400003AA300001135000046A30000E4
:10AB6400153500004FA30000193500005AA300005A
:10AB74001D35000065A30000FD3400006EA3000035
:10AB8400C534000077A30000D5340000D0A3000032
:10AB9400B9440000DCA30000D3440000E2A3000099
:10ABA40003450000E8A3000087440000EEA3000072
:10ABB40041420000F8A300003545000000A4000055
:10ABC4006D4300000DA40000C14500001BA400005B
:10ABD400C545000024A40000C945000029A40000C4
:10ABE400CD4500002EA40000D14500003AA4000089
:10ABF400D545000041A40000D94500004AA4000046
:10AC0400DD4500004FA40000E14500005AA4000007
:10AC1400E545000064A40000BD4500006EA40000EA
:10AC2400B945000003000000020000000800000015
:10AC34000A000000FFFFFFFF000000000100000009
:10AC44000000020001000000FFFFFFFF0000000001
:10AC5400020000000000040002000000FFFFFFFFEC
:10AC640000000000030000000000080003000000D2
:10AC740000000000E8A9000008AA000028AA0000BB
:10AC840000000000000000000000000000000000C0
:10AC9400ACA800000000000000000000000000005C
:10ACA40000000000000000000000000000000000A0
:10ACB4000000000000000000000000000000000090
:10ACC4000000000000000000000000000000000080
:10ACD40020020020E7A800003901000075470000A9
:10ACE400954A0000916200000D0100000000000080
:0400000300005E5D3E
:00000001FF
